:020000041100E9
:10300000002373B52B4D2C4C28006361022601F080
:103010006DF94021FE2221742800284B009601F012
:10302000B7F9002836D1217CFF222800244B0096D6
:1030300001F0AEF900282DD1224BA2899A4226D167
:10304000E389214A93420DD1204B6361204B2268D2
:10305000002A03D1002B01D043CB43C4280001F048
:1030600083F973BD1B4A934201D00023EFE71A4B4B
:103070001A4A1B68934206D9C02304222800217CE7
:103080009B0001F0FBF9114B6361154BDFE7002357
:103090002374EAE7CC233821AC2228009B01217459
:1030A00001F0ECF90028F2D10E4B63610E4BE38185
:1030B0000E4BCCE7A442FF1F7062FF1F7C62FF1F14
:1030C0007E62FF1F5959000083050000194100115D
:1030D0002CBD0011821500009462FF1F87130000B1
:1030E00038BD0011D1410011AAAAFFFF20BD001177
:1030F000F7B5164B0192C318021D002000938823D8
:103100005B05D3181B685C1C1AD09CB2402C18D8E5
:103110008D781E0CAC466746CD782D023D43AE42FD
:1031200006D1019800280ED110000C70240A4C70B2
:1031300003249BB20733A343D218009B9A42DED3E9
:10314000FEBD4432F9E71000FAE7C046FC0F00006C
:10315000802213B503000324019189B25201073183
:103160009B18A14304305A1A88235B05C3181B68B7
:10317000591C03D190429241104016BD99B240298A
:1031800007D80B000733A343C0189042ECD30020AC
:10319000F3E74430F9E7134B134A1B68126810B584
:1031A000FA24934201D81A00F824104BE4021B6859
:1031B0009A4210D813000E4A12689A420ED3013375
:1031C00007D1F823DB029C4203D10A49054808F0E5
:1031D0002BFD200010BDFC24E402ECE7FE24E402F9
:1031E000F7E7C04600C0071100D0071100E0071143
:1031F00000F00711FFFFFF7FF0B59BB015000490B2
:103200000391402A00D9A0E006AB59801A80FFF74D
:10321000C2FF0400042816D9002206A9FFF768FFA0
:10322000052810D906AB1B88AB420CD1002D07D066
:10323000514B2A000499C01808F08EFB002802D1D7
:1032400001201BB0F0BD06AB1D8020000699FFF7E2
:103250007FFF041E7BD1069B0793FFF79CFF802313
:103260005B01C618802307001B039E4201D3F8268A
:10327000F60288235B05F31801931B68013302D023
:10328000019808F0A1FB3D49019808F0CDFC3B1DD9
:103290000293331D05938822029B52059B181B68DD
:1032A00008935A1C3CD044219AB20091402A04D879
:1032B0000320D11D814389B2009103991B0C8B42DD
:1032C00024D0402A22D80122300008A9FFF710FF9D
:1032D000021E1BD1380008A9FFF70AFF04000428CA
:1032E00031D9009A059B9B1880225201B218934253
:1032F00040D288235B05C118009A09A808F0E4FBB6
:103300001D4B009A09A9F01808F016FC009A029BC0
:103310009446634402931A4B029AFB189A42BAD31A
:1033200088235B05FC1821680198013908F07CFCB2
:10333000200008F049FB039A07AB5A803000079938
:10334000FFF706FF0400002C03D1002079E70428D2
:10335000FBD988235B05E018069908F065FC032378
:10336000EA1C9A4300D16BE7034B0499E01808F07C
:10337000E3FB65E70424ECE704000011FFFFFF7F97
:10338000F80F0000F7B505001400402A21D80027E7
:1033900001AE71803780FFF7FEFE042816D93A008F
:1033A0003100FFF7A5FE042810D93688BC420BD0A7
:1033B000BD4209D0221CB44200D9321C064B92B245
:1033C000C118280008F080FB30B2FEBDC04300B237
:1033D000FBE703204042F8E70400001137B5042260
:1033E00004000D0001A81649FFF7CCFF02000428D5
:1033F0000BD1019BA34208D3AB4204D0104901A8D2
:103400000195FFF7F9FE01203EBD0E4C2368200018
:10341000019308F0D9FA019920000139019108F0CF
:1034200003FC80235B01E418074B9C42EED104228D
:10343000034901A80195FFF7DFFE0020E4E7C0463D
:103440005555000000C007110000081130B589B0C3
:1034500008F09AF910226946254808F08DFA254BA4
:10346000009A9A420ED1019B029A0F2B33D8002169
:1034700001240698013B08D2002900D00292029B49
:10348000013331D10023029325E0551CF2D1020013
:103490002100EFE710341022200004A908F06CFA94
:1034A000029B013301D1069B0293882304995B059B
:1034B000C918059B06981A03120B049105928142C4
:1034C00003D02B4201D108F0FFFA019B013B01938D
:1034D000019B002BDED1029B002B03D004930498A8
:1034E0004168084709B030BDE025014C2D03EFE7E6
:1034F00000000111504859368022F8B5964C974B80
:10350000D200002120001C6008F016FA2300944A23
:1035100088331A60934B1A786A23002A00D011333B
:10352000E3620A232365904B37221B780820A363AC
:103530008E4B2118E361102323628D4B3B25636181
:10354000C823DB00A36123008C331A602823013ACF
:10355000E26320646364CA67043A211DCA672100DC
:10356000BC310D602100C03108602100C4310B6006
:1035700021000635CC310D602100083DC8310D60B9
:103580002100D0310A602200D43210602200D832EB
:10359000136022000227E032210017604222DC3152
:1035A0000A6021001B3DE4310D602100E831086014
:1035B0002100EC310B6023000521F4331960230056
:1035C000F0331A602300183290331A6023009433CA
:1035D000186023001E3A98331A60AF23DB00236083
:1035E000644BFA262363644B644DE360644BF03113
:1035F000A3642300FF31FC33B600A16021611E608B
:10360000A5627325E5656D3D6565A56596255D4AF1
:10361000AD00E264666258606766A566002709250A
:10362000A767E566584F594D606720002567E26738
:103630003A6015279C30676007001A203860200028
:10364000A0300700212038602000A83007004C4837
:1036500038602000F830066026006427A436376002
:1036600026005F3FAC3637602600033FB036376038
:103670002600C637B436376026000027B8363760D4
:1036800038269E60424E96205E64424E5A66DE6147
:10369000414E9A645E62F53EFF3E9E621E269A6728
:1036A000354A8000DE661F675F67DD651D6618624C
:1036B000DA67BE23394A5B00E250394BD8382350D1
:1036C00004302250C4225200A350C623E4205B00E1
:1036D000E1500433334AE1503349344BD16034492B
:1036E000800019503349E938FF3819503249043005
:1036F000195032493248D16132491163324951631C
:103700001900F4310860CE20304940001160304982
:10371000195019002F48F83108602F49D1658221CE
:103720002E4A89005A501A002D490832D1671A00D2
:103730002C49B432116088212B4A89005A501A0052
:103740002A49883211602A4ADA6408F02DFA0120E9
:1037500007F082FFF8BDC0460004FF1F1465FF1F7D
:10376000F06FFF1FE044FF1F4A0AFF1F3A070000E7
:1037700080C3C9019A020000DC0500006A1800003D
:1037800050C3000088130000F009FF1F204E000006
:103790006509FF1F68100000C409000040420F00C7
:1037A00010270000FC00FF1F751CFF1F0000FF1FFB
:1037B000C92CFF1F5930FF1FF12EFF1F3520FF1F9F
:1037C0002527FF1F5120FF1FFD21FF1FC11FFF1FC6
:1037D0004929FF1F312AFF1F8D19FF1F5528FF1F81
:1037E0007925FF1F8525FF1FC11EFF1F791FFF1FA2
:1037F000391EFF1F0223F0B50124614D614E2B706D
:10380000614B91B01C70614F039333680021082015
:10381000FB7006F0EDFD082006F0E4FC0023984262
:1038200005D0FA78552A02D0332A00D09BE03360C5
:10383000042006F057FF08F007F8FFF75DFE08F0D8
:1038400023F81F2201240021514B10AE1A70514B56
:103850001C70514B1970514B19689143163A0A4329
:103860001A60602219689143403A0A431A6008F0CE
:10387000E3F908F0D9F8C120FF21494B80001A581C
:103880008A431A50C522920098588843BF39014391
:1038900099509858434908408021C901014380202C
:1038A00099509958C0050902090A0143995080218D
:1038B0003D48490108F030F8032322003B490194B8
:1038C00000933B4807F098FE2C223A4905A808F0DF
:1038D000FBF805AC61782078023406F0A3FCA64220
:1038E000F8D1354C0020012106F0B0FD2268334BA1
:1038F00003201A40A023DB021343236080232268A5
:103900009B041343236022682D4B1A4080239B03A2
:10391000134323602B4A2C4B934200D8012007F01D
:1039200083FE07F0F1FE80232268DB04134323604B
:10393000287807F089FE039B1878C0B207F0CCFE08
:1039400007F09AFF2149042007F04EFE06F096FE8C
:1039500000F03EF800F0E8FD00F090FE00F00AFAFA
:10396000002011B0F0BD00932100184A042008F097
:10397000C3F88023DB059C62FFF768FD58E7C0466B
:103980004A0AFF1F34F00040E044FF1FA062FF1FFF
:10399000480AFF1F490AFF1F680AFF1FBCF00040CA
:1039A00000E100E0FF00FFFFE444FF1F6857FF1F36
:1039B000E454FF1F48BC001114F00040FF7FF8FFE3
:1039C000FFFF9FFF0080FF1FF06FFF1F3B000108FC
:1039D000002210B51100112007F0B6FF10BD000045
:1039E000F8B500230926374F374C3B62E3681120B6
:1039F000B343E36008F008F9112007F005FF112038
:103A000008F0CAF8402322688025134323608023EE
:103A10006268DB0213436360A3682C4A2B43A360F4
:103A2000A36802211340A3608023A2689B01134373
:103A30001022A360236C072093432364236C0F3A66
:103A40001343236480235B003B62226B204B1A40AC
:103A50002263626B1A406263A26B1A40A263E26B3C
:103A60001340E363E3681B4A1340E36006F0DAFBAC
:103A70000121072006F0EAFC174B11205A6C154370
:103A80005D6407F0B1FEFD21144B154A89005A50C0
:103A90008023C720626B5B0313436363E36880008A
:103AA0003343E3600F4B104A195811408022120231
:103AB0000A431A50802292051A6008220B4B5A635F
:103AC000F8BDC04600F000403CF00040FFFFDFFFC3
:103AD000EFFFEFFFFFFF7FFF003800400000FF1FF8
:103AE0005118FF1F00E100E0FF00FFFF000005404C
:103AF00070B5284C238C002B23D0228A002A21D198
:103B0000DA0023826382A382E38223836383A38315
:103B1000E38322606260A260E2601F4D1F4A64205E
:103B2000EB8093420AD8FA220020D200934205D9B2
:103B30001B4A0A21981807F0F7FDC0B2002328722B
:103B4000238470BD0720E11CCA7F01320240CA777E
:103B500005D10325201DC17F01312940C1770832DD
:103B60005200A352002321001A00088A01321B18B8
:103B70000231082AF9D1221DD27F9200A350626837
:103B800023689B18A2689B18E2689B185B099BB28C
:103B9000C3E7C046E061FF1F8862FF1FB70B00004C
:103BA00030F8FFFF30B503A804880B20002C0ED19D
:103BB0004968074D08784978090201430A20A9425B
:103BC00005D1012120001980024B1B7A137030BDF2
:103BD000192A00008862FF1FF7B5150008AA168889
:103BE0004A680F4F14785278120222430A24BA42CC
:103BF00014D10122DBB2019200962A0007F08EFC5C
:103C0000041E0BD1074B1B68002B07D068782A785D
:103C10000002104342425041013098472000FEBD4F
:103C2000022900000C62FF1F30B501250379040052
:103C3000BFB02B4211D00A49408806F0DBFF284272
:103C40000BD0084B01A95B8D4D800B80064B0022E9
:103C50001B7A60880B7104F0ADF83FB030BDC046F0
:103C60000462FF1F1841FF1F8862FF1F10B505493E
:103C7000054806F075FF0421044A054806F032FFA6
:103C800010BDC0460462FF1FFFFF000074BC00119E
:103C90001841FF1F10B5024804F00EFF10BDC046CA
:103CA000293C0011012303700B4B1A7A4270022247
:103CB00082709A78C270DA780271032242711A799E
:103CC00082715A79C2710C2202729A794272DB793E
:103CD00083720B207047C0468862FF1F022310B515
:103CE0000370013B43700533837010330371443B11
:103CF00043712A3383714433C37100230372064B2B
:103D000004001B8843720A30FFF7CCFF831D0A3082
:103D1000C0B2E37010BDC0468862FF1F10B514200A
:103D200007F082FD124B14220021186007F004FEF8
:103D3000002007F059FF012007F066FC022007F081
:103D4000EBFE032004F05CF9042006F071F9052075
:103D500003F09AFB062004F067F8072001F06AFAE6
:103D6000082006F09FFE092001F036F810BDC0467D
:103D70001062FF1F07F078FD012007F035FE07F005
:103D800073FC0000094B10B50400984205D00129CE
:103D900004D12000064906F0E3FE10BD0229FCD143
:103DA000013904F047FE0028F3D0F6E7FEFF0000DB
:103DB0003662FF1F70B50D7A100004AA2C00168819
:103DC00010221440154220D1002E20D10A78022A58
:103DD00018D14A68517815780E4A09022943914250
:103DE00005D00D4A914209D01C800A2404E0142217
:103DF0000A491A8007F068FE200070BD0C220849AD
:103E00001A80F7E71C800124F6E70824F4E70B2466
:103E1000F2E7C046F3FF0000F4FF00006C43FF1F11
:103E200050BD001110B504000749084806F098FE7F
:103E3000074804F081FD0020E40704D50721054A66
:103E4000054806F04FFE10BD3662FF1FFFFF000061
:103E5000853D0011B8BC00115C41FF1F00B50C4B43
:103E6000BFB01A780B4902A800F0C2FC6B4680B2C2
:103E7000D880002809D06A46074B01A91B88938087
:103E8000064B0022188803F095FF3FB000BDC046E6
:103E90001462FF1F1562FF1FB641FF1FC042FF1FC4
:103EA00000B50C4BBFB01A780B4902A801F0C8FE50
:103EB0006B4680B2D880002809D06A46074B01A91A
:103EC0005B8D9380064B0022188803F073FF3FB090
:103ED00000BDC0463E62FF1F3F62FF1F5C41FF1FE7
:103EE000C042FF1FF7B50E00377A1C0008AB110067
:103EF0003D001A8820231D401F423CD13378022BFD
:103F00003BD173681F785B781B023B431E4FBB425B
:103F100008D01E4FBB4214D01D4DAB4221D00A2504
:103F20002800FEBD002A2AD1142C2AD82200F068CD
:103F300007F0CAFD174B1C70012CF1D9FFF7B0FF39
:103F4000EEE7002A1BD1202C1BD82200F06807F0D6
:103F5000BBFD114B04211C70104B187807F02CFD91
:103F6000DEE7E3B20124009201940A00310007F079
:103F7000D5FA0500D4E70825D2E70125D0E70B25BF
:103F8000CEE70D25CCE7C046F3FF0000F4FF0000AC
:103F9000022900003E62FF1F1462FF1FC062FF1F64
:103FA000332310B5040003700A220749013007F0DB
:103FB0008BFD064B0F201B681A0AE37222731A0C42
:103FC0001B0E6273A37310BD8862FF1FB062FF1FD8
:103FD00030B5012503790400BFB02B4213D00B4943
:103FE000408806F007FE28420DD06A46084B02A81A
:103FF0001B889380FFF7D4FF6B46D880002260882F
:1040000001A903F0D7FE3FB030BDC0463662FF1FA6
:10401000B641FF1F10B5024804F04EFD10BDC0466A
:10402000D13F001170B5160004AA148805AA1578AE
:104030004A685078117800022A4A084380180528F7
:104040004BD807F081FD03131E29343F0720032CB2
:104050000BD80422121BAA4200D92A0022491A8036
:104060003000091907F030FD002070BD0720112C29
:10407000FBD81222121BAA4200D92A001B491A801F
:10408000EEE707200E2CF0D80F22121BAA4200D90F
:104090002A0017491A80E3E70720032CE5D80422F9
:1040A000121BAA4200D92A0012491A80D8E7072019
:1040B000032CDAD80422121BAA4200D92A000E4986
:1040C0001A80CDE70720032CCFD80422121BAA4266
:1040D00000D92A0009491A80C2E700220A201A8062
:1040E000C3E7C046DCD5FFFF03BD00115C62FF1FC4
:1040F000F3BC0011EEBC0011E9BC0011E4BC0011DE
:1041000010B50D21024A034806F0ECFC10BDC04674
:10411000D8BC0011CC41FF1FF0B50024274E85B05C
:104120003000B47100F0E2F8254D264BEA89297C75
:104130009A422FD10423300003AA00F057F904005B
:10414000300000F011F90123B371002C34D16B461B
:1041500099892B68C9BA4B4329891B4A1B145B18E0
:1041600053806B46D9896B6849BA89B24B436989D8
:104170001B0C5B181548191C1BB2834200DD011C87
:104180000B0400D500211388918001331380200097
:1041900005B0F0BD0227220003AB3000009700F00D
:1041A000F7F80E230400297C0122300000976B44AD
:1041B00000F0EEF80443C3E71C00E8E7A442FF1F49
:1041C0007062FF1F830500008862FF1F0F27000039
:1041D00073B5234E300000F089F8224D07236A465C
:1041E0003000297C00F002F904003000002C33D1AB
:1041F0006B461B787F2B2FD800F0B6F86B46D8782B
:10420000F02302041B031A406B469B8816495BBAD5
:104210009BB21A432B68000953432A891B0C9B1835
:104220004B806B465A789B7812031B011A436B68CC
:10423000024353436A891B0C9B180C481A1C1BB27F
:10424000834200DD021C130400D500220B888A8003
:1042500001330B80200076BD00F086F80124F9E7D9
:10426000A442FF1F7062FF1F8862FF1F0F2700001C
:1042700070B5114C237C002B0FD0382B0ED10F4D75
:10428000280000F033F8CC23AC222800217C9B01CD
:1042900000F0F4F8280000F067F870BD084BE289E0
:1042A0009A42FAD1054D280000F020F8002228009B
:1042B000217C00F0C5F8EDE77062FF1FA442FF1FEC
:1042C0008305000010B5084B1A7C002A09D05B69F1
:1042D000002B06D09847041E01D0FEF791FE200067
:1042E00010BD0124F9E7C0467062FF1F70B5C179A7
:1042F00005000C00631E9C411A4BE402E4184900BF
:104300000460C9B2007906F0D7F8E9796879490004
:104310000131C9B206F0D0F8E8790930C0B207F02F
:104320003BFC0023E36661332360AA795B3B002AF0
:104330000ED022689A43023B134323600A23E361B1
:104340000733236200232363A3630133E36370BD58
:1043500022689A4302231343236046236361063392
:10436000A361EFE70050004070B50025040003682A
:10437000DD66C0790930C0B207F046FC290020791B
:1043800006F036F82900607906F032F870BD0000BA
:10439000F8B51E0006AB1D78002304681700E3661D
:1043A000616007F0F1F901238022E3662B002761A9
:1043B0005200013B08D207F0A7FB08200A4A116807
:1043C000002D03D12800F8BD2261F2E7236F0342DC
:1043D00003D02369013D3370013613685B1A032B48
:1043E000EED90125EEE7C0466008FF1F70B51C003E
:1043F000002305681600EB66696007F0C5F9012324
:104400008022EB6623005200013B08D207F07CFBC0
:1044100008200A4A1168002C03D1200070BD2A61CF
:10442000F2E72B6F034203D02B69013C3370013656
:1044300013685B1A032BEED90124EEE76008FF1F17
:10444000002370B504681500E366616007F09CF90D
:104450000123E366256107F057FB8020064A8000B0
:104460001168636B034205D113685B1A032BF8D9FB
:10447000012070BD0020FCE76008FF1F70B51D0023
:10448000002304681600E366616007F07DF90123EC
:10449000E36626610F33626B1A42FCD02B0A23615C
:1044A0001023626B1A42FCD0EDB2256107F02CFBA1
:1044B0008020074A80001168636B034205D11368AE
:1044C0005B1A032BF8D9012070BD0020FCE7C04621
:1044D0006008FF1F70B51E00002305681400EB661E
:1044E000696007F051F90123A619EB660F33B44256
:1044F0000ED107F009FB80200A4A800011686B6B1F
:1045000003420CD113685B1A032BF8D9012070BD4C
:1045100021782961696B1942FCD00134E7E700205A
:10452000F5E7C0466008FF1F10B5084CE368002B94
:1045300008D18022064B52021B689B186360054B12
:104540001B68236007F028F9A06010BDB062FF1F50
:10455000C8F00040CCF0004070B5184A936A916AE8
:104560009942FBD116498A689A421FD39A1A8B60E6
:10457000144B0126186893B2D202D20E4343424331
:1045800000204C681B0A1B1912029B180E4C0A686B
:104590004B60551CA3420CD8002801D04B600A6028
:1045A0000A4A136008680A4B186070BD581E821AC8
:1045B000DDE7084A30009B182A00EAE700F00040D7
:1045C000B062FF1F140AFF1F40420F00C8F00040F6
:1045D000CCF00040C0BDF0FF70B51F4C23793F2BDD
:1045E00001D93F2323711D4B22791A701878C0B26C
:1045F00007F0A2F818231A491A4A0B801A491380A7
:104600000B805380A379194980200B800C21938063
:1046100001334B43164D191C0001834200D9011C84
:104620002980D1806379002B11D101336371237A02
:10463000012B01D8022323726279237A0D48534358
:104640000A21584307F070F80B4D286070BDA02B6D
:10465000EDD9A023EAE7C046A462FF1F480AFF1F66
:10466000BE42FF1F8C44FF1FBC42FF1FBA42FF1F08
:10467000B842FF1F710200009462FF1FF8B51421B9
:104680000020FEF7ABFE114C011E114D09D10C228A
:10469000104BC1CBC1C4280007F04EF9FFF79CFFB7
:1046A000F8BD0C2220000C49FEF76CFE0C2802D04D
:1046B000084B43CB43C40C2228000849FEF762FE96
:1046C0000C28EBD00C220021E5E7C046A462FF1FB6
:1046D0007062FF1F44BD0011FC0C0000F50C0000CF
:1046E000F0B51D4C8022A544040088206946520183
:1046F000400506F0D1FF902212016A441300200009
:1047000032C832C316C816C38023144C144FA6688F
:104710009B033343A3603B6007F026FA8823A0681D
:104720005B05C01807F050F9002588232900802276
:10473000A0685B05C01840196944520007F0FCF9F5
:1047400080230135FF355B019D42EED1A6603E60BE
:10475000044B9D44F0BDC046FCEFFFFFFC43FF1F30
:104760009808FF1F04100000F0B5040087B000286F
:1047700025D0684607F010F91B4C022806D1062206
:104780006946200007F0E8F8002816D069460023A3
:1047900001250F262F00E25C0133100910308740FD
:1047A00038002F00324097403A0002434A610439F2
:1047B000062BEFD16846FFF793FF07B0F0BD182234
:1047C00069460A4806F068FF6A46A300D3580133D9
:1047D00005D01822FF21684607F0AEF8EAE7013459
:1047E000062CF1D1E9E7C0466509FF1F0009001159
:1047F000F0B5002504000E0085B0AA4200D186E085
:104800004B1C087801934B78897837790902194352
:10481000F3783F061B040B431F430397207065701A
:10482000252800D196E033D8112813D807F064F872
:1048300069002501250125012501AA00B800B10064
:104840002501250125012501250125012501250138
:1048500005011F01232800D1DEE0DB2800D02EE176
:10486000042A00D8ACE01025052A05D0551F2A00DF
:104870003800711D07F028F905223100200007F0EB
:1048800023F92A003900601D07F01EF905353EE0C6
:10489000562859D010D8332800D19DE0552839D05A
:1048A0002628DAD19C4B2900132218001D0007F09E
:1048B00043F8FEF7A5FB5CE0712800D177E0722891
:1048C00000D180E0602800D18BE0DC28C5D1022A2D
:1048D00000D875E07378BFB26370B378A370032A11
:1048E00005D0033A390092B2F01CFEF785FC102285
:1048F0003900E01CFEF746FDC51C002807DA607091
:104900005CE00C222000854907F0DEF80C25280029
:1049100005B0F0BD013A824D0C2A13D8002A0AD006
:104920002800019907F0D0F8FFF756FE0C22280066
:104930007C49FEF761FC29000C22601C07F0C4F8DA
:104940000D25E4E70C22EBE7754D774B2A0043CBAE
:1049500043C2E9E7013A704D0C2A11D8002A08D069
:104960000199280007F0B0F80C2228006F49FEF7E3
:1049700043FC29001322601C07F0A6F81425C6E7A3
:104980000C22EDE705226A49601C07F09DF8062518
:10499000BDE712226749601C07F096F81325B6E7B9
:1049A00008226549601C07F08FF80925AFE7717888
:1049B000F02905D8614B188801F09EFD0225A6E775
:1049C000FF236370FAE75E4B012A03D072789A7076
:1049D0006270F3E79B78F4E72000FFF7E1FA050047
:1049E00095E7013A564B574D062A10D8002A10D0A9
:1049F000012128005970019907F066F801F052F87A
:104A000029000622601C07F05FF807257FE70622D1
:104A1000EEE700225A70F3E7042A04D94A4D2F60CA
:104A200006F0BAFEA860FFF797FD0422039003A9E1
:104A3000601C07F049F8052569E7444D062ADFD9CF
:104A400006222800019906F087FF0028D8D0062208
:104A50000199280007F038F806223D492800FEF7A2
:104A6000CBFB0123364A91780B439370C8E7012AA8
:104A7000A6D07078FFF778FEA0E7012800D0ECE61A
:104A8000931E344F132B04D87378002B09D100F0F8
:104A900015F9314B39001D78601C6A1E07F014F8B7
:104AA00035E7551E2A000199380007F00DF82B490B
:104AB000AAB23800FEF7A0FB00F038F9E9E7DA28DF
:104AC0001DD1042A00D87BE7082A15D9B379727959
:104AD0001B021343F27912041A43337A1B06134361
:104AE0003B603B68052231002000039306F0ECFF99
:104AF0000422601D03A956E7FE236370F1E7DE2858
:104B000000D05DE7511E012A01D10025FFE6019882
:104B100000F0AEFFF9E7C0467062FF1F50BD001104
:104B2000A462FF1FFC0C000044BD0011F50C000046
:104B30007C62FF1F5C62FF1F0044FF1FC042FF1F1B
:104B4000A062FF1F5D43FF1FB062FF1F6509FF1FCB
:104B5000ADAC0000A164FF1F9F64FF1FAEDE00002C
:104B600070477047020010B5094B0A32094C92B2E7
:104B7000DA815A8298811882207802F023FB04227D
:104B8000054B012120781A7006F016FF10BDC046B3
:104B90008A43FF1FEA64FF1FE964FF1F013870B5F5
:104BA000042809D806F0D0FF030928081200234B77
:104BB0000221187806F000FF70BD204B08211878FC
:104BC00006F0FAFF00221E4B1A72F5E7802200243D
:104BD0001B4B1A4D52001A8108211A682878DC7282
:104BE00006F06AFD2100287806F0C6FF012000F0DB
:104BF00077FE00F057FFDFE7104B0821187806F02A
:104C0000DBFF1048FFF76AF80F4B104A9B79002032
:104C100093800F4A13808022094B5200D8721A8168
:104C200000F05EFE00F03EFF0A4B9B78002BC3D0E5
:104C3000094A136006F030FEBEE7C046C062FF1F9F
:104C40009462FF1FC942FF1FA462FF1F8C44FF1F15
:104C5000BA42FF1FA062FF1F34F0004010B50129C7
:104C60000BD1082809D1054B1B78002B05D0262233
:104C7000034B04485A72FFF775FF10BDC264FF1F53
:104C80009462FF1FC40900000300F0B50A4D8E189E
:104C9000B14202D152008018F0BD0C782F6824096F
:104CA0003C5D0F271C700C7801313C402F683C5D47
:104CB0005C700233ECE7C046B442FF1F0D22124B7A
:104CC00010B51A700C23114C11492370093A033B9B
:104CD0001048637006F0F8FE2D2301220E490F489C
:104CE000A371FFF7D1FF01220D49FFF7CDFF01228C
:104CF0000C49FFF7C9FF030000200B4902001870A0
:104D0000FEF77AFA10BDC046BE64FF1F9F64FF1F06
:104D100003BD0011A164FF1F6709FF1FA664FF1FE9
:104D20006609FF1F6509FF1FAEDE000070B5124C5B
:104D3000142220001149FEF725FB431E104D132BB2
:104D400017D8AB78002B14D0431C2B7009236B7041
:104D5000002300190370287829000130C0B206F042
:104D6000BBFE297822000139C9B2002005F0D8FD28
:104D700070BDFFF7A3FFEEE7A164FF1FAEDE0000EA
:104D80009F64FF1F10B5114B1A781870002A0ED0BF
:104D900000280BD10E4B1A78062A07D85423D3408B
:104DA000DB0703D50B4B187802F00CFA10BD002876
:104DB000FCD0074B1B78012B02D0033B022BF5D80C
:104DC000044B0121187806F0F7FDEFE7C264FF1FDE
:104DD000E964FF1FEA64FF1F70B5514E514A524902
:104DE0003070082005F028FC0121022005F02EFB80
:104DF000022005F00FFC0121002005F027FB002018
:104E000005F008FC00F0B8FEFEF7FAF806F01CFE0C
:104E1000032246494648FFF737FF2D2403000422AA
:104E20001C7044490130FFF72FFF30230470424DBE
:104E3000424C437083702E3B062220004049EB8792
:104E4000FEF7A0FA062813D0200006F0A5FD0228E0
:104E500009D00321200006F00FFE8D23E3706E3B86
:104E6000237119336371062220003549FEF7C4F916
:104E7000344B1B68FC335C64FFF758FF0020FFF7DE
:104E800081FF314C314A0121314B1278207802F0F8
:104E90005BF9304A304B12780021207802F054F947
:104EA00001222E4B1A702E4BDB78552B31D12D4B16
:104EB0003B325A722C4B2D4AAB81EA812B826A829B
:104EC0002021307806F0B8FC0120404205F074FD46
:104ED0000120404205F010FEFFF712F9FEF7C6FE72
:104EE00000F0B2FC01204042FEF79CFF012006F0DA
:104EF000B3FDF02001F0E4FA0121307806F05CFD0A
:104F0000307802F0BBFA1A4806F0CEFBFEF768FDD7
:104F100070BD6422174B5B7953431A000A32CBE70A
:104F2000C062FF1F614B00115D4C00110044FF1F68
:104F30005C62FF1F7C62FF1F8A43FF1F6509FF1F22
:104F4000ADAC00001465FF1FEA64FF1FE842FF1FBD
:104F5000C942FF1FBE64FF1F9F64FF1F9064FF1FB5
:104F6000A062FF1F9462FF1FC4090000CE09000069
:104F7000C262FF1FA462FF1FF8B50A0020230D00C4
:104F80001A40194263D05E4B1B78002B5CD0FFF7B0
:104F9000E3FA5C4B5C4C5D4E99686268737A8A1ADE
:104FA000DB039A4202D36160FEF71AFD327A217A5E
:104FB000531EDBB2994205D1FFF75AF9002000F0E9
:104FC000A7FD15E09142F9D300272772FFF77AF980
:104FD000A37ABB4202D0A772FEF78AFD012000F03F
:104FE00097FD4B4F3800FEF779FE390006F0CCFCF8
:104FF000637A002B25D0013BDBB26372002B20D1FA
:10500000444BDB78552B01D106F046FCE37A002BAC
:1050100012D00023A27AE3729A4202D0A372FEF762
:1050200067FD3D4A3A4F1388380001331380FEF77D
:1050300055FE390006F0A8FC642370795843FFF749
:1050400091FD237A0133237220206840F8BD0BB212
:10505000002B0ADA314B187806F0B6FB002801D095
:1050600006F0DAFD80200002EFE70224214206D09C
:10507000254B01201A72FFF785FE2000E5E70B079C
:105080001ED5FFF769FA1F4B1F49204C98684A68E4
:10509000637A821ADB039A4202D34860FEF7A0FCCF
:1050A000FFF710F9FFF7E4F8012000F031FD00F000
:1050B000E5FB2368DB0701D5FEF7ACFF0820C4E75A
:1050C000CB0609D5FEF714FD0D4B1B78002B01D143
:1050D000FEF7E0FD1020B8E70124214207D0104878
:1050E00000F06CF806F000FB00F0F8FCC5E70424C3
:1050F000080020402142A9D0FEF7B0FEBDE7C0461F
:10510000C264FF1FB062FF1F9462FF1FA462FF1FF3
:10511000C942FF1FA062FF1F8862FF1FC062FF1FFE
:10512000AC42FF1FF0B51B4B1B4F1B883A88040095
:105130001A4E1B4D85B09A420DD832889A420AD336
:10514000184B1A882B889A4205D1174A174B128898
:105150001B889A421BD0052001F008FA3B8802AA5E
:1051600013803388019053802B88114D93800F4B0F
:1051700002A91B88D3800F4B2A78188802F024FFDD
:105180000D4B08212878019A1C7006F00DFB05B024
:10519000F0BDC0468E64FF1FBE42FF1FBC42FF1F12
:1051A000BA42FF1F8C64FF1F8A64FF1FB842FF1FB3
:1051B000EA64FF1FC042FF1F8864FF1F13B50C4B3A
:1051C0001C78002C11D1002801D00A4B18600A4A23
:1051D0000A4B11780A4A10780A4A01920A4A009248
:1051E000002205F095FA200016BD1124FBE7C04609
:1051F000E964FF1F8464FF1FE864FF1FD864FF1F7A
:10520000EA64FF1FC464FF1FC864FF1F10B5064B8C
:1052100012201B78052B06D1044B13221988044B4E
:10522000187801F07FFB10BDE964FF1FC042FF1F2B
:10523000EA64FF1F10B500240122114B524218707E
:10524000104B1C70104B1A8002F018F904220F4BFF
:1052500021001A700E480C3206F0EEF910222100DF
:105260000C4806F0E9F907220B4B1C600B4B1C7035
:105270000B4B1C700B4B1A700B4B1C7010BDC046B7
:10528000EA64FF1FE964FF1FC042FF1FE864FF1FBD
:10529000D864FF1FC864FF1FC464FF1F9E64FF1F04
:1052A0009D64FF1FC242FF1F9C64FF1FF8B5174C8F
:1052B0000600257806A814240078052D23D1B41FF4
:1052C000134FA5B21824BD421DD88D1FADB2BD42EB
:1052D00019D8FA256D00AA4215D21D000D4F0A3DBE
:1052E000ADB2BD420FD80C4C26800C4C21800C492D
:1052F00000240A800B4A1380FFF714FF0A4B042195
:10530000187806F059FC2000F8BDC046E964FF1F7C
:10531000790C0000750C0000BE42FF1FBC42FF1F4D
:10532000BA42FF1FB842FF1FEA64FF1FF0B50BB27D
:105330000D0089B0002B00DB70E1A44E307806F040
:1053400043FA041E50D00378A22B00D122E1D02BC7
:105350001AD0912B45D143780E2B42D19C4B828899
:105360009A423ED19B4A83681278052A39D103209C
:1053700018567F2835D0984B1B68002B31D05B68BE
:10538000002B2ED098472CE08078072829D806F0EB
:10539000DBFB0428183F3F74A8D86378002B0CD19E
:1053A00001218C4B19708D4B1A78002A5BD08C4BE5
:1053B000307801F0C9FE002855D00722854B1A70BD
:1053C00051E061780029F8D1E378002B11D0854AAB
:1053D000854B1278307801F0B7FE60706378002B4F
:1053E000EBD1200006F018FC80200002684009B0D4
:1053F000F0BD784B1B78022BF3D00121307806F0FA
:10540000DBF90028EAD10121307806F0D5FAE5E78A
:105410006378002BD1D16F4F032807D13B78052B40
:1054200002D101333B701EE00223FBE76F4B1A8869
:105430006F4B0293002A0BD01B78002B03D0012165
:10544000307806F0B1F93B78062B04D1013BE9E74F
:10545000029B1A70F7E7042B41D10121029B30789F
:10546000197006F0A9FA5C4B1B68002BB9D01B68B9
:10547000002BB6D0574A107884E76378554F002B3D
:1054800027D10622211D5B4806F01EFB62895A4B7C
:105490005A491A80A2895A4B1A80E3890B80052148
:1054A000397058490A80584A1380228A574B1A800B
:1054B000574B1B78012B09D11F2001F057F8FA2216
:1054C000920042430421307806F06EF90022484BE6
:1054D00075E7312B00D070E70022454B1A7003238B
:1054E000A0E706220021434806F0A6F80023454A1B
:1054F00004211380444A30781380444A138006F014
:105500005BFB0821307806F057FBA379083B5A4231
:105510005341304A03331370304B1B78002B06D0B5
:10552000334B30781A78002A06D001F04BFE012266
:10553000314B52421A8096E70121197006F03CFA6D
:10554000F5E70821307806F037FB6378002B00D0B0
:1055500047E72C4B2D4F0293E388029A04211380D6
:10556000294B307803932389039A138063893B8006
:1055700006F022F9002800D033E7264B1B68002BE9
:1055800000D12EE7039902983A88098800881B68A1
:10559000984726E74379132B00D022E70389012B94
:1055A0000AD11D4B1B78022B06D10821307806F05A
:1055B00003FBFFF72BFE14E7052000F0D7FF0821BF
:1055C0000200307806F0F0F80BE7C046EA64FF1FEF
:1055D00005140000E964FF1F8464FF1FE842FF1FF9
:1055E000C942FF1FBE64FF1F9F64FF1FC064FF1FEF
:1055F000C264FF1F9164FF1FC042FF1F9864FF1F1A
:105600009A64FF1F8E64FF1F8C64FF1F8A64FF1F54
:105610009064FF1F8064FF1F8864FF1F8020C0010B
:10562000014200D0E2E6CB0731D5324B1B78002B8C
:105630001DD0314E05AC3378052B1AD1023B2370B7
:105640002E4B21001B7823722D4B1B7863722D4B40
:10565000187801F01DFD002809D007202A4B307072
:105660001B68002B03D01B68002B00D0984701203B
:10567000BCE60E20254B06221B7825492370254BBE
:105680001B78637002ABC01806F01EFAD8E702233D
:1056900008001840194209D0174B1B78052B03D17D
:1056A0001D4B188806F040F902209FE60424214291
:1056B00003D0FFF737FD200098E6082308001840C4
:1056C000194200D193E6154B1C78012C03D0022C13
:1056D0000DD008208AE6124B124A134913481B8842
:1056E0001288098800880094FFF7E0FDF1E7FFF7D2
:1056F0008DFDEEE7C264FF1FE964FF1FC242FF1F7A
:105700009C64FF1FEA64FF1F8464FF1F9E64FF1FE9
:10571000C342FF1F9D64FF1FC042FF1F8864FF1F1D
:10572000B842FF1FBA42FF1FBC42FF1FBE42FF1F0D
:1057300010B502A804880B20002C10D14968087805
:105740004978090201430C48814209D1022119809C
:105750000A4B59881170DB7800205BB2537010BD82
:10576000074C0A20A142FAD102211980034B9988E3
:1057700011705B79F0E7C0466E2A00008862FF1F57
:105780006F2A0000F7B5150008AA16884A680F4F5F
:1057900014785278120222430A24BA4214D1012208
:1057A000DBB2019200962A0005F0B8FE041E0BD170
:1057B000074B1B68002B07D068782A78000210433B
:1057C00042425041013098472000FEBD02290000AE
:1057D000FC64FF1F30B5012503790400BFB02B42E4
:1057E00025D01449408805F005FA28420CD0124B08
:1057F00001A95B8D00220B8002234B800F4B5B883D
:105800008B80608802F0D6FA0D49608805F0F2F9C5
:10581000C0070CD50B4B01A91B8800220B8002236B
:105820004B80064B9B888B80608802F0C3FA3FB0A8
:1058300030BDC046F464FF1FEC42FF1F8862FF1FAB
:10584000EC64FF1F4643FF1F10B5074C07492000BB
:1058500005F086F92000064905F082F90721054A7E
:10586000054805F03FF910BDFFFF0000F464FF1F7D
:10587000EC64FF1F70BD0011EC42FF1F10B5024821
:1058800003F01AF910BDC046D557001170B55F2559
:10589000082607498400CA788B7840012A40B34320
:1058A0003440A843234302438B70CA7070BDC04686
:1058B0005D43FF1F010043B204205A0002409B00D9
:1058C0000C3003401A43152310B5044CE07898437C
:1058D000143B0B4018430243E27010BD5D43FF1FB1
:1058E00010B5054B082419790A00A243002801D0FD
:1058F00022000A431A7110BD5D43FF1F10B5054B0E
:105900004024D9780A00A243002801D022000A438B
:10591000DA7010BD5D43FF1F0821F8B5324D334BDF
:10592000AE7804000E40AE70984204DD67232B7001
:10593000473B6B70F8BD2E4B984203DAE0232B7087
:105940003A3BF6E700232B706B7083B21A002948AC
:105950005F3292B2284F82422CD9002C03DA5B428C
:105960001CB204232B70053420B20A2105F0DCFEA2
:1059700004B2FA239B009C4232DB08232A781343AB
:105980002B706421200005F0CFFE0A2100B206F042
:105990008BF809B22A787B5C13432B700A21200014
:1059A00005F0C2FE0A2100B206F07EF809B27B5C67
:1059B0006A780AE06970002CDBDA5B421CB20423CF
:1059C0002B70F3226B78092CE8DC13436B700A21EF
:1059D000200006F069F809B27B5C1E43AE70A9E7AF
:1059E000632CCEDCEDE7C0465D43FF1F1B4E00007D
:1059F0001DFCFFFF2A0800009ABD00110823F7B51F
:105A0000194FCD003E7904001E403E71EDB263286F
:105A100006DD5F3333433B7120231D437D71F7BDAA
:105A20000300093305DA20235B4233433B71A6238D
:105A3000F3E70E4B019300280BDA0423444224B20F
:105A40003B710A21200006F02FF8019B09B25B5C34
:105A5000E3E70928F5DD0A2105F066FE019B00B2A7
:105A60001B5C1E433E71ECE75D43FF1F9ABD0011B6
:105A7000F8B50A4F05003B780E00002B0CD0084CFF
:105A80002000FEF733FC33002A0020003978FEF7AF
:105A900021FD2000FEF768FCF8BDC0460765FF1F2A
:105AA0006443FF1F70B50A4E0A4D062231002800DC
:105AB00005F052FF002809D0074C310006222800CB
:105AC00006F002F807212000FFF7D2FF70BDC046A4
:105AD0005D43FF1F0165FF1F0065FF1FE622402198
:105AE00010B50A4B1A70403A5A703E329A70DA7802
:105AF0000A40DA70082219791140053A0A431A71EE
:105B000047225A71FFF7CEFF10BDC0465D43FF1F0D
:105B100010B500282AD0164C0A210223E05E05F0B9
:105B200003FE00B2FFF7F8FE0423E05E642105F0F7
:105B3000FBFD012100B2FFF761FF237A002413224D
:105B400020009A426041C0B2FFF7D8FE0320FFF761
:105B50009DFE2000FFF7AEFE064B18780538434245
:105B60005841C0B2FFF7BCFEFFF79CFF10BDC04616
:105B70008862FF1FE964FF1F70B500250A4C2000F2
:105B8000A571FEF7B3FB10233E212000074AFEF764
:105B9000A1FCA84200D13E35054B20001D70FEF748
:105BA000E3FB0123A37170BD6443FF1F8ABD001195
:105BB0000765FF1F0200F0B501270A480A4E511879
:105BC0008B1A002B00DCF0BD0824157843086840D0
:105BD00038404000805B013C58406D08002CF5D1F6
:105BE0000132EDE7FFFF0000AABD0011F0B500256E
:105BF0000F269D4200DBF0BD4C5D07094440344058
:105C0000A400A05801357840F3E70000F0B589B052
:105C10006A460D000B000F27110010351C78013368
:105C2000260024093E40167054700232AB42F5D172
:105C30002023024AFFF7DAFF09B0F0BDB0BD001122
:105C4000F0B54E780B7889B036020C001700019041
:105C50001E43012A61D9954B9E4200D877E001335B
:105C60009E421CD1062A17D1CA788B7812021A4399
:105C70000B791B0413434A7912061A438C4B5A6161
:105C800000221A705A808B4A5A608B4A9A608B4A5B
:105C9000DA60002009B0F0BD88225205EEE7884B9B
:105CA0009E423CD182498B78002B00D0F6E00C2A32
:105CB00031D10F22A3789343E27812021343227961
:105CC000120413436279120613434B60E279A07900
:105CD00012020243207A00041043627A1206024341
:105CE000CA60E27AA07A1202024376484A8183426D
:105CF00008D804236E49142201980B7005F0E4FEC5
:105D00001420C7E71201D21889235B059A42F0D804
:105D100001238B70BDE7022AFAD00523EAE76A4A1D
:105D200001239642E6D1FFF771FA052F0CD9E378EB
:105D3000A2781B021343227912041A4363791B06CB
:105D40001343624A0393136005F0A6FDA1E7584D83
:105D50002B78002B9DD1AB78002B00D1A0E02B89B4
:105D600001339BB20093B34200D091E0132AD4D9FF
:105D7000CF7C8B7C3F02122120001F43FFF71AFFCC
:105D8000874200D08EE0002E3DD1E378A2781B023E
:105D900013432279E96812041A4363791B061343FB
:105DA00003930A228B4212D1FF23A370E370237165
:105DB00063716B89002B09D1E37B227C1B021204E7
:105DC0001343A27B13431B0901336B8100226B89B0
:105DD000002B8ED0002A67D1686837013818000B75
:105DE0006B6900030390984205D9686105F0ECFDEA
:105DF000EB780133EB7068681022A11C381805F0AD
:105E00009BFE2E8145E76F89009A7B1E9BB29342D1
:105E10003AD1E278A37812021A43237905A81B0429
:105E2000134362796C6812061A43EB68009203927E
:105E3000211D0C22049305F047FE0120260004A931
:105E400040421036FFF7E2FE013F012F17D1009AC2
:105E50000B232861824200D04CE704221C49200019
:105E600005F06AFE042203A9686805F015FCE968DC
:105E7000039AFF23914200D13CE7F73B3AE7310018
:105E8000FFF7C4FE1036DFE70923B742A4D831E795
:105E9000009BB34200D9FCE607232BE7022329E746
:105EA000032327E7062325E70A2323E7FFFE000055
:105EB0006C43FF1F00000111FFFF000050485936DE
:105EC00001FF0000FFFF001102FF000034F000405E
:105ED0007843FF1F10B5034C0B000122210000F096
:105EE0006BFA10BD956000110B8870B506000D00AF
:105EF0000224162B11D92B000322094900F05CFA69
:105F0000041E0AD1074B2A881B88191C934200D90A
:105F1000111C300089B200F0EFFA200070BDC046BD
:105F2000C16000112E65FF1F10B54A780400013AC8
:105F30000B000220012A07D80A78002A04D0052283
:105F40002000024900F038FA10BDC046EF60001191
:105F50000A7810B50B0004000220002A04D00722A2
:105F60002000024900F028FA10BDC0469B610011D4
:105F70000A7810B50B0004000220002A04D0092280
:105F80002000024900F018FA10BDC046016200115D
:105F900010B5034C0B000B22210000F00DFA10BDD0
:105FA0003162001110B5034C0B000D22210000F0EE
:105FB00003FA10BDA362001110B5034C0B000F22B1
:105FC000210000F0F9F910BDFD6200110A7810B54A
:105FD0000B0004000220002A04D0112220000249F4
:105FE00000F0EAF910BDC0460D630011002310B5A2
:105FF0001322190000F0E0F910BD000010B5034CA9
:106000000B001722210000F0D7F910BD5F630011CB
:10601000002310B51922190000F0CEF910BD0000C0
:1060200010B5034C0B001B22210000F0C5F910BD78
:1060300099630011F7B584890D0006000121002C39
:1060400022D000238268D3561778002B1EDA0C2C3E
:106050001AD90C3CA4B2131940880093230002F013
:1060600086FE431E984101307B06DB0F6B703F2399
:10607000013C1F40A4B22870AF70AC80002C07D048
:10608000B3680133AB6000210800FEBD0020EBE7E0
:10609000AC60F8E70B7803704B8843704B881B0AA1
:1060A00083700B79C370042070470420022B06D143
:1060B0000020537811781B02009A0B43138070471D
:1060C0000B8803700B881B0A437002207047042062
:1060D000009983420AD1537810781B0203430B8046
:1060E000D37890781B02034300204B807047F8B5AB
:1060F0000D004B7801240021461C03702B788B4245
:1061000001D82000F8BD6B78B01C4F1C012B10D1BA
:10611000890069184B88022233704B88B9001B0A2A
:106120007370691805F020FB04360434A4B2F9B288
:10613000E4E7122359436B185A88043132705B88A4
:1061400010221B0A7370691805F00EFB1236123408
:10615000ECE770B5049D14001E00052B01D8042047
:1061600070BD637812781B0213432B80E378A2780A
:106170001B02134302226B802A71211D681D063EFB
:1061800005F0F2FAB2B22A81E92AE8D82800A11D66
:106190000A3005F0E9FA0020E2E7002310B50A789A
:1061A0009A4201D8900010BD9A008A185488013391
:1061B00004705488DBB2240A4470948884709288F6
:1061C000120AC2700430EAE710B51100029C062BD7
:1061D00004D004201022142B01D010BD0222227101
:1061E0004B7808781B0203432380CB7888781B0206
:1061F000034363800431601D05F0B6FA0020ECE72C
:1062000010B50C788B7804315C43E4B20370220043
:10621000013005F0A9FA601C10BD0420022B06D144
:106220000020537811781B02009A0B4313807047AB
:1062300010B50C000A88023105F096FA208810BDCE
:1062400070B504000D0004981100012B01D8042042
:1062500070BD167852781202324302800200F13289
:1062600055701470E125002C00D10C35023B9AB218
:106270004280AA42EBD80231043005F075FA0020C2
:10628000E6E70420009983420AD1537810781B0274
:1062900003430B80D37890781B02034300204B808C
:1062A000704710B50C000A88023105F05DFA2088AD
:1062B00010BD000070B501211E000420049C0E409A
:1062C0000B4218D1CB40DDB28D4214D90A49DBB262
:1062D000098899420FD32300EE331D703300580014
:1062E00011184978165C0902314301332152D9B2A1
:1062F0008D42F4D8002070BD8443FF1F10B50C0000
:106300000A88023105F030FA208810BD10B50C78EB
:106310008B7804315C43E4B203702200013005F055
:1063200023FA601C10BD10B511000298032B01D890
:10633000042010BD14785278043B120222430280DC
:10634000CA788C781202224342809AB28280EB2A69
:10635000EED80431063005F007FA0020E9E710B561
:106360000C000B8803700B881B0A43704B888370EA
:106370004B881B0AC3708A880430063105F0F4F993
:10638000A088043080B210BD0420012B03D100206E
:106390001378009A1370704710B50C000B880370C7
:1063A0000B881B0A43704A880230043105F0DCF97F
:1063B0006088023080B210BDF0B589B003931E4BE7
:1063C000029242000700D05A019102F020F81325F2
:1063D000061E2DD0029B01240370019B002B04D0CC
:1063E000001903999847001984B26B461B7A5BB277
:1063F000002B0FDA1021380002F01CFB19250028B1
:1064000013D130003219E1B202F066FC051E0CD146
:106410000C34A4B2042304AA380005A9938006967C
:10642000948101F0AFFD051E02D0300005F0F4F9B3
:10643000280009B0F0BDC0462C65FF1F70B50500EF
:106440000C0000280CD00020814209D0102220002E
:10645000044905F089F901202B7823736B78637365
:1064600070BDC046F0BD0011F0B506000D0017006C
:106470001C0085B002291BD00020102907D1022B57
:1064800007D0102B03D115E00020102C08D005B048
:10649000F0BD69463800FFF7D1FF2A0069460BE0DE
:1064A00069463000FFF7CAFF22006946380004E061
:1064B000022BE9D12A003900300005F0ADFAE6E7F9
:1064C000031CF02800D9F023032008499AB2013AAE
:1064D0000B80D317034006499B189B100B80D30FEA
:1064E00004499B185B100B807047C0468843FF1F10
:1064F0008643FF1F8443FF1F034B1B888B4202D33D
:10650000024B4000C15270478843FF1F2C65FF1F9C
:10651000014B4000185A70472C65FF1F1722014B92
:106520001A8070472C65FF1F70B505000E2005F01E
:10653000DBF9041E13D0D0230370002306228370DE
:1065400007494570033005F00FF9064B2100DA8A40
:1065500062811B7E2373044B187805F085FA70BDA9
:106560004865FF1F3865FF1FD843FF1F262803D843
:10657000024B4000C05A70470148FCE78A43FF1FA6
:10658000FFFF000070B506000C00094D1C22002121
:10659000280005F051F8074B1E70074B1C7005F0E2
:1065A0002BFB0123002801D0002312202B7070BD8B
:1065B0003865FF1FD843FF1F5965FF1F70B50500E1
:1065C0000D4C0800E260A16010220021656005F01A
:1065D0006BF9012803D11021A06802F058FD1022A8
:1065E0000021280005F060F9012803D1102160681E
:1065F00002F04DFD70BDC0463865FF1F70B5041E2A
:1066000005D1002903D006220D4805F0ADF80D4B49
:106610001D78012D11D1002C05D102221A7005F030
:1066200033FA280070BD00221A70074B1B78FF2B2D
:10663000F7D02000FFF778FFF3E70025F1E7C04629
:106640004865FF1F3865FF1FD843FF1F030010B5C3
:10665000002801D1002010BD00780B4A002803D18A
:106660005988D1821B7913761378022BF2D100233B
:10667000984200D103331370044B1B78FF2B01D0D9
:10668000FFF752FF0120E6E73865FF1FD843FF1FE1
:10669000002911D000280CD04B79012803D14022C9
:1066A0005242134303E03F221340032802D001204B
:1066B0004B7170474022F4E70800FAE770B5094DC6
:1066C0000100287800280BD0074C0622200005F096
:1066D0004BF821002878FFF7DBFF200005F03CF89D
:1066E00070BDC0465865FF1F3265FF1F00290AD0E4
:1066F000012808D13F224B799343C02B03D0403B64
:106700005A425341981C704770B5174D06002B78BC
:10671000FF2B15D00A2005F0E7F8041E10D0D02377
:106720000370C83B8370114B11491B784670C370CE
:106730000622043005F018F82100287805F094F9B5
:106740000C4B1B78012B0DD10B4B1B68002B03D07E
:106750009B68002B00D09847084B04211878084A02
:1067600004F0AAFF70BDC046D843FF1F5865FF1F45
:106770003265FF1F5465FF1F8065FF1F8465FF1F83
:1067800060EA0000014B98687047C0463865FF1FFB
:10679000014BDB68186870473865FF1F074B10B561
:1067A000DA68136801331360054B1878FF2803D0AB
:1067B0008021C90105F000F910BDC0463865FF1FF2
:1067C000D843FF1FF7B50E0002F0C8F8051E1CD015
:1067D0000E4B06621F78002F00D10778AB7910208E
:1067E000019305F081F8041E0FD0D0230380C73B2E
:1067F0008370019BE91DC3700622043004F0B4FFCE
:1068000021003800E66005F02FF9F7BDD643FF1FE1
:10681000014B18787047C0465865FF1F054B00288C
:1068200005D1054B1A78054B002A00D1014B180001
:106830007047C0464865FF1F5865FF1F3265FF1F40
:10684000014B58687047C0463865FF1F024B1868F7
:10685000431E9841C0B270475C65FF1F421E030093
:106860000120152A03D9FF3B5A425341D8B2704741
:10687000F0B51C0000230E0085B0039002920B704F
:10688000029A934201D3002019E0E55C5A1CD2B26F
:10689000002DF8D0029851198142F4DC0233DFB2A6
:1068A000A35C18000193FFF7D9FF002807D0013D32
:1068B000019A0399EBB233708A4202D1E01905B014
:1068C000F0BDDB19DBB2DBE710B50C0002F09EF87F
:1068D00003001220002B03D02100588805F064F833
:1068E00010BD000070B50E4D84006359002B15D00B
:1068F000186A002801D005F067F92B59586A00285A
:1069000001D005F061F92B59986A002801D005F0F3
:106910005BF9285905F058F900232B5170BDC0468A
:106920006865FF1F1C4B70B504000E0015009942EE
:106930000AD11A4B1B68002B01D1122070BD1B68B5
:10694000002BFAD09847F9E7154B994215D1134B14
:106950001B68002B0AD01B68002B07D09847002823
:1069600004D1104B1C70104B1D70E7E7290020006C
:10697000FFF7AAFF0028E1D1F3E7080001F0EEFFDE
:106980000028DAD003780320A342D7D129003000B1
:1069900005F00AF8D2E7C046FEFF00006465FF1F5D
:1069A000FFFF00006165FF1F6065FF1FF7B5040072
:1069B000808801F0D3FF0025A84203D00578A08885
:1069C00002F008F81C4E3378002B1FD0AB421DD1CB
:1069D0001A4B28001978FFF777FF002818D00023FA
:1069E0003370A3790820A778A688019304F07CFF70
:1069F000011E0DD0D0230370CA3B8370019B4770EA
:106A000086808371280005F02FF801E0002DE8D181
:106A1000A0880B4B8200D358002B01D0FFF762FFF8
:106A20001721A088FFF768FDA08801F027FDA08846
:106A300001F0FEFDF7BDC0466165FF1F6065FF1FE9
:106A40006865FF1FF0B587B01D000CAB1B88070001
:106A500001930DAB1B88142002930EAB1B8816000C
:106A600003930FAB1B880091049310AB1B88059315
:106A700004F03AFF041E1AD0D0230370CB3B4770BA
:106A80008370C670062229000430002D11D004F056
:106A90006BFE019B21006381029B0098A381039BF5
:106AA000E381049B2382059BA37404F0DDFF07B000
:106AB000F0BD04F0C1FDECE7F7B5009308AB1B880F
:106AC00007000C200D001600019304F00DFF041EBA
:106AD00013D0280001F042FF00280FD00078D02307
:106AE0002370C93BA370009B21002381019B677029
:106AF000A580E680638104F0B7FFF7BD014B1878ED
:106B0000EDE7C046D843FF1F13B50400648903892D
:106B1000C2888188C0780094FFF7CEFF13BD0000C3
:106B200010B5044C2068002803D005F04DF8002370
:106B3000236010BD6C65FF1FA122F0B58188920013
:106B40004A43384B384F1B6804009B189D22920023
:106B50009B18827989B01A603B68002B5FD01D7842
:106B6000324B1B68002B04D05B68002B01D0002047
:106B70009847260008363100E079FFF7B7FD237DFE
:106B8000E0710200E0780493638A29000393238A6A
:106B90000293E3890193A38800933300FFF752FF28
:106BA000E378002B0BD1E289A379A18802920196A8
:106BB000E27928000092012201F0DAFEE0703B68E1
:106BC000002B20D0FFF7ACFF194D287800281AD0F1
:106BD000184B1978FFF778FE002814D02B78E67848
:106BE00008200793A78804F07FFE011E09D0D02358
:106BF0000370CA3B4670837087808671079804F0E3
:106C000033FF00232B701721A088FFF775FCA088A5
:106C100001F034FCA08801F00BFD09B0F0BD064B7B
:106C20009DE7C0463409FF1F6C65FF1F8065FF1F8D
:106C30006165FF1F6065FF1FD843FF1FF8B50700A0
:106C400008000E0001F08AFE041E18D02620FFF76F
:106C50008DFC051E00D12578062004F045FE041E9B
:106C60000DD00021062204F0E7FCD0232370C23BA4
:106C700021006770A370A680E8B204F0F5FEF8BDAD
:106C8000F0B585B001930AAB1B78070002930BABFC
:106C90001B7808000D000092039301F05FFE061EB2
:106CA00022D0102004F020FE041E1DD0102200214E
:106CB00004F0C2FC2620FFF759FC002800D13078F0
:106CC000D0232370C13BA370009B21002372019B42
:106CD00067706372029BA580A372039BC0B2E372CC
:106CE0000C9BE36004F0C0FE05B0F0BDF7B50D00ED
:106CF000019001F033FE071E20D00E2004F0F4FDB9
:106D0000041E1BD02620FFF731FC061E00D13E7862
:106D1000D0232380C53B0622A370F91DE01C04F09C
:106D200023FD019B2A0063810123DD401A401D40A1
:106D3000210022736573F0B204F096FEF7BD0000E7
:106D4000F0B585B0029010000D0017000A9E039365
:106D500001F004FE041E31D0029B002B2ED1039BB8
:106D600002795B0724D5122313430422002E08D195
:106D70000B99002905D10C99002902D10D99002900
:106D80001AD01A430D9B2271002B00D0C9E0002EAF
:106D900000D1CFE0002D00D0CCE0606A002801D007
:106DA00004F012FF1C21300004F0B6FC606205E024
:106DB00002239A430E33D7E793432371654BBA00FE
:106DC000D458002C00D1AAE0002E10D0236A002B4A
:106DD00003D11C2004F028FD20625E4BBA00D3587A
:106DE000186A002803D01C22310004F0BDFC0C9B63
:106DF000002B12D0574CBB001D596B6A002B03D1DE
:106E0000162004F011FD6862BB00E358586A0028A0
:106E100003D016220C9904F0A7FC0D9B002B11D077
:106E20004C4DBC006659B36A002B03D1142004F00A
:106E3000FBFCB0622B59986A002803D014220D99EC
:106E400004F092FC380001F089FD051E67D0414B2B
:106E5000BA00D358002B62D01A6A3420002A00D11D
:106E60001C389A6A002A01D0143080B20B9A002A8A
:106E700001D01C3080B25B6A002B01D0163080B28A
:106E800004F032FD041E4AD01822002104F0D4FB85
:106E90002620FFF76BFB0190002801D12B7801938E
:106EA000D0232370029B200063700A23294EA37015
:106EB000039BBD00A371AB59A780196A1830002944
:106EC00005D01C22A06004F04FFC20003430735920
:106ED000996A002907D0030014221433E06002935A
:106EE00004F042FC02980B9B002B08D003001C22EC
:106EF0001C330B992061029304F036FC02987359FD
:106F0000596A002903D01622606104F02DFC6B46FB
:106F10002100187904F0A8FD3800FFF7E3FC05B064
:106F2000F0BD10220D9B0D991B69A018236204F07F
:106F30001BFC2CE70B9B002B00D13FE7012D00D061
:106F40003CE7606A002801D004F03EFE1C210B984B
:106F50002AE7C0466865FF1F10B5044C206800286A
:106F600003D004F031FE0023236010BD5C65FF1FD9
:106F70000B4B07B51A68002A01D100200EBD6946E7
:106F8000531C012012780731FFF772FC0028F4D05F
:106F900002780123100018401A42EED0EEE7C046F6
:106FA0007865FF1FF0B51F4F01203B6887B0002BAD
:106FB00025D09B78059300F0B3FB002821D00A2050
:106FC000FFF7D4FA04000B20FFF7D0FA164B0500A8
:106FD0001E78731E9E413B68F6B2191DD878FFF7E4
:106FE00057FB3B682900DA7A043303929A790193BC
:106FF0000292009033002000059A04F095FD07B03E
:10700000F0BDFFF7B5FF002805D00620FFF7AEFA68
:1070100004000720D8E70820FFF7A8FA0400092099
:10702000D2E7C0465C65FF1F5865FF1F70B50A4E6A
:10703000040033780D00FF2B0DD0042004F054FC25
:10704000011E08D0D0230370CE3B45708370C470FE
:10705000307804F009FD70BDE843FF1F70B50400EF
:1070600006200D0004F040FC011E0AD0D02303705E
:10707000CD3B8370054B44701B688580187804F005
:10708000F3FC002C01D0FFF767FF70BD5C65FF1FAC
:10709000F8B5264F06003B680D001124002B05D1E2
:1070A0000522234B1B78134202D112242000F8BD85
:1070B000204A10241268002AF8D01278002AF5D04D
:1070C000DB0719D52B789A1E012A1AD80C2004F058
:1070D000ABFB132438600028E8D000230A22437059
:1070E00029000670023004F03FFBFFF75BFF041E2F
:1070F0000AD0FFF731FFD9E700F012FB0028E1D1F9
:10710000E4E7002BE2D0D0E70B4B1B78032BCDD16B
:107110001D20FFF72BFA094B18800028C6D0084B1A
:1071200004211878074A04F0C7FABFE75C65FF1F1F
:107130005965FF1F7865FF1F5865FF1F5665FF1FC4
:107140008465FF1F60EA0000F7B50193194B140036
:107150001A78052306000F0012201A4221D00129B7
:1071600020D1154B1D68002D1BD002201F2C18D8D4
:10717000002C02D0019B002B13D0104B1F221E703D
:107180006E1C0021300004F057FA019922003000F3
:1071900004F0EAFA310020002C70002F06D004F031
:1071A000ABFAFEBD064B12201D68DCE704F094FC30
:1071B000F7E7C0465965FF1F7865FF1FE843FF1FCB
:1071C0007465FF1FF8B50F4E12243368002B17D0DB
:1071D0001B780F3C834213D100250B4F02213878D6
:1071E00004F0EAFC094B042138781D8004F0E4FC2B
:1071F000074B28001D8033685C7004F05DFC0400C0
:107200002000F8BD5C65FF1F8465FF1F7065FF1FD0
:107210005665FF1F70B5012823D11B4C2388002B16
:1072200003D01A4A1578002D07D0194B1B68002B84
:1072300002D01878FFF7C6FF70BD3B2B02D93C3B4C
:107240002380F9E7134E0221307804F0B5FCFA22CE
:107250002388920002215A43307804F0A5FA258051
:10726000EAE70B4B1B68002BE6D00B4B1B785B0748
:10727000E2D5084B0221187804F09EFC0022024B54
:107280001A80FFF769FED7E77065FF1F5465FF1F7F
:107290005C65FF1F8465FF1F5965FF1FF8B51E4D14
:1072A0002868002803D004F08FFC00232B601B4EBD
:1072B0003068002803D004F087FC00233360184FA7
:1072C00005243B7818002040234221D0154800F0C7
:1072D0002BFA3B78234213D0202004F0A5FA286033
:1072E000002813D02022002104F0A6F9202004F069
:1072F0009BFA041E306005D02022002104F09CF986
:10730000002004E0286804F05FFC2C601320F8BD26
:1073100000F00AFAF4E7C0467865FF1F7465FF1FA6
:107320005965FF1FDC43FF1F10B50A4C23681A1E66
:107330000ED0002808D10130587004F0BDFB0028A1
:1073400005D02368002B02D00021FFF787FE012221
:10735000100010BD5C65FF1FF7B5274E05003368B0
:107360000191181E21D05C78244F012C30D1FFF7F9
:10737000FFFD002825D02000FFF7F8F80400412881
:1073800014D91F4B022118781E4A04F095F91E4BA0
:107390003C3C1C80022233685A703B78002B14D18D
:1073A00028000199FFF75AFE0120FEBDFA22920043
:1073B0004243002AEED0124B0221187804F0F4F96F
:1073C000E8E7FFF7D3F80200F3E700233B70EBE7B1
:1073D0003B78002BE8D1032004F086FA011E08D088
:1073E000D0230370CC3B457083703368187804F069
:1073F0003BFBFFF7B1FDD7E75C65FF1F5465FF1F3F
:107400008465FF1F60EA00007065FF1F10B5174913
:10741000838802008B4220D011D815498B4217D0A7
:10742000144900205B1899B2012907D89268117895
:107430005A425341D8B2FFF7F9FD012010BD0E4A60
:1074400000209B1807229BB29A424041C0B2F5E748
:1074500083681878FFF768FFF0E7836899785A78AF
:10746000090218781143FFF777FFE7E70A200000C9
:1074700006200000F8DFFFFFAFDFFFFF014B1870B1
:107480007047C046E943FF1F10B5064C207001F05D
:1074900041FA207804F0E0F90521207800F062FD3F
:1074A00010BDC0468465FF1F0BB273B50D00002BE5
:1074B00000DBC4E0884B187804F086F9041E0ED077
:1074C0000378912B0FD0A22B00D1A1E0834B187829
:1074D000FF2852D0210004F0C7FA00284DD18020A7
:1074E0000002684076BD43780F2B76D013D8052B69
:1074F00070D00E2BEAD18088794B98422BD8794BEB
:1075000098421BD8784B9842E0D1A3681878591C50
:10751000FFF774F838E03E2BD8D18378032B74D072
:107520006CD8012B6ED0022BD0D1704B1B68002B76
:1075300023D05B68002B20D098471EE06C4BC0180E
:107540000C28C3D804F068F81DC2C2150BC20B0B7F
:107550000B3223C23C00674BC0180728B6D8664BD5
:107560001B68002B09D01B68002B06D02000984711
:107570000AE0A3681878FFF7C7F8200004F04CFB76
:10758000ADE7A068FFF762F800289FD0F5E7A36891
:107590001B78002BF1D0554B1B68002BEDD01B68DE
:1075A000002BEAD0210055489847EDE74F4B1B6868
:1075B000002BE2D01B68002BDFD021005048F3E7FE
:1075C000504B1B68002BD8D05B68002BD5D0210016
:1075D0004348E9E7FFF7EAF9CFE780884A4B98424A
:1075E00003D04A4B984200D070E7464B1B68002BF3
:1075F000C3D05B68002BC0D02100D5E7153B012B21
:10760000BBD963E7FFF798FAB7E7FFF77DFAB4E76E
:107610003F4B1B78042B07D100236A461380017966
:10762000408800F0C5FCA8E7364B1B68002BA4D0AF
:107630005B68002BA1D00100364898479DE70124E4
:1076400021420AD0294B1B68002B04D05B68002B19
:1076500001D000209847012043E78B070AD5264B2D
:107660001B68002B04D05B68002B01D020009847DA
:10767000022036E70421280008400D4200D131E7FE
:10768000254E3388002B21D0013B9BB23380002B49
:107690001AD1FFF7DBF800280AD0204B1C70164BDC
:1076A0001B68002B04D05B68002B01D0200098479A
:1076B000FFF7C6F8694601F001FD6846FEF7FEFFD8
:1076C0001D20FEF753FF308004200AE7024B187894
:1076D00004F072FAF8E7C0468465FF1FE943FF1F14
:1076E0000E20000001200000091000007C65FF1F33
:1076F000FEDFFFFFAFDFFFFF8065FF1F0C200000F4
:107700000B2000006465FF1F0D2000001320000007
:107710005965FF1FFFFF00005665FF1F5465FF1FDF
:1077200010B501F09BF910BD014B18607047C046C1
:107730008065FF1F0B880020162B01D8172304201B
:10774000014A13807047C0462E65FF1F0020704716
:10775000074A03001188814207D09188002099428E
:1077600002D101308000101870470020FAE7C046AF
:107770008C65FF1FF0B58F7806000D00C5B01E2F79
:1077800015D1FFF7E5FF051E03D10024200045B009
:10779000F0BD00223B003100C078009200F0B2FB47
:1077A0000400A81C00F0D2FBFF23EB70EEE7264B91
:1077B000062403931B78FF2BE8D0182FE6D87B080C
:1077C000224A013BDB0002929A589446002ADDD0FF
:1077D000029AD3185B68002BD8D00878002802D111
:1077E0004B78012B02D10624122FCFD107AFAB88E3
:1077F000697800976446AA68A047041EC6D1AB7892
:10780000029A5B08013BDB00D318390030005B684B
:107810009847041E0BD1AB78042BB6D0039A3100E5
:1078200010782200009700F06DFB0400AEE76A7844
:10783000002AABD1AA7805A93B88087130000A70EC
:107840004B80FEF747FBA0E7EC43FF1F00BE001193
:107850001D4B37B5050098420BD000290AD1FFF720
:1078600077FF002805D11948FFF772FF002800D0E4
:10787000058037BD01291AD1FFF76AFF041EF8D031
:1078800001235B420380A378FF2BF2D0FE2B07D0AD
:107890000023E0781422009329001E3300F032FB0D
:1078A000A01C00F053FB01235B426380E1E7022947
:1078B000DFD1013901F0BEF80028DAD12800FFF746
:1078C00047FF041EDFD1D4E7FEFF0000FFFF0000EA
:1078D000022210B5074B52421A80074801325A80E3
:1078E0009A80DA8000F07EFA044801F025F8002042
:1078F00010BDC0468C65FF1F7577001151780011CF
:107900000388F7B50400002B02D102252800FEBD34
:1079100042680221137825485268FEF7A5FD002829
:107920002ED0234F01253A88002AEFD080232188CA
:107930005B0201259B1A9942E8DC0C2003F074FFDE
:10794000061E31D03B8822889C46002318000195F2
:1079500061469DB2491989B2AA421BD8002801D0BC
:1079600062443A8000233000082208C0210003F05E
:10797000FBFE104A1368002B13D100251660C5E7E3
:107980006268022113780C485268FEF76DFD0028EA
:10799000C7D1BAE760681D014019418101330198E0
:1079A000D6E71A001B68E6E71325AFE76EBE0011A5
:1079B000EA43FF1F8865FF1F6CBE0011014B187062
:1079C0007047C046EC43FF1F14230A0010B51A404D
:1079D000194204D00122102101F048F810BD4B06D5
:1079E000F9D4012088434000F8E710B514008B0655
:1079F00004D50122102101F039F810BD08230A0036
:107A00001A40194202D14BB2002B0FDA102101F0BB
:107A10002DF8002808D02300F2331B78002BECD07F
:107A2000F1342378012BE8D10020E6E70320890711
:107A3000FAD4E2E7F0B51F00184B85B01C6801903E
:107A400002910392002C27D1200005B0F0BDA5685B
:107A50003301ED186B89019A934211D3029A934234
:107A60000ED8002F04D10A9B002B10D12C00EBE77D
:107A70003B002978039A6868FEF7F6FC0028F2D1EB
:107A80000136B6B2A388B342E1D82468DAE7A36826
:107A90000A9A5B891380E9E70026F3E78865FF1FF0
:107AA00037B50C000A8849880123914217D3002A70
:107AB00015D0651D23792A0002210A48FEF7D4FC5F
:107AC000102300280BD023796188208800242A0005
:107AD0000094FFF7AFFF0A23A04200D02300180054
:107AE0003EBDC0466EBE001113B50A000888498825
:107AF000012388420BD8002809D0002413790532CD
:107B00000094FFF797FF0A23A04200D0230018003B
:107B100016BD13B50A0008884988012388420BD88E
:107B2000002809D00024137905320094FFF782FF62
:107B30000A23A04200D02300180016BDF0B58BB078
:107B400003904A8808880E000123824255D30028FA
:107B500053D00023012704AC237000227188130046
:107B60000092FFF767FF051E3ED02078002835D130
:107B70002B78022B18D167706A8983000130E318D3
:107B800080005A8069680222201803F0EDFD2378F6
:107B90000133DBB22370042B19D93B006889013013
:107BA00080B2002BD9D01FE0022363701223584308
:107BB0006A89231804305A8069681022201803F05B
:107BC000D3FD23780133DBB22370002BE5D10C4ABF
:107BD0006B899B185A425341DBB2DFE76378012B74
:107BE000E4D12B78022BC7D022780A23002A04D0B4
:107BF00021000398FEF798F9002318000BB0F0BDA0
:107C00000100FFFF0F4BF0B504001868002816D0E4
:107C100083685D89A54207D88288AE18B44203DA2A
:107C200012019A18934201D10068EFE71E005F89A4
:107C30001036A74204D1002900D00D801800F0BDF5
:107C40003300EFE78865FF1F70B505000C0008885A
:107C50000021FFF7D7FF03000120002B04D02200F2
:107C60002800197AFFF7C1FE70BDF7B50C0000259A
:107C700001902300EE331B78AB4201D800200AE0CC
:107C80006B00E65A00213000E718FFF7BBFF002821
:107C900002D126800130FEBD017A0198FFF794FEE3
:107CA000002802D03B882380F5E70135EDB2E0E7FC
:107CB00010B5040008880021FFF7A4FF030001208D
:107CC000002B03D02000197AFFF77EFE10BD0000C4
:107CD000054B1B68002B01D1180004E09A685289FB
:107CE0008242F6D1988870478865FF1FF0B50E274D
:107CF000002687B0039302ABFF183E8005001F4BA0
:107D000040891400984207D02B78013000976A68A8
:107D100080B2FFF78FFE060002212B7818486A68B0
:107D2000FEF7A2FB00280FD06C892000FFF7D0FFE0
:107D3000002802D0013C0419A4B2039B002B00D000
:107D40001C80300007B0F0BD02212B780D486A6816
:107D5000FEF78AFB0028E7D102212B780A486A68DF
:107D6000FEF782FB002807D0002EDED03B88A3421E
:107D7000DBD17489013CDFE76C89DEE7FFFF00009F
:107D80006EBE00116CBE00116ABE001110B50C0071
:107D9000FFF7DEFC03000220002B0AD0002C00D0ED
:107DA00023609B781720FE2B03D00138FF2B00D1D6
:107DB000002010BD73B50D0001A904001600FFF7E7
:107DC000E5FF172805D0002E04D129002000FEF77A
:107DD00027F976BD01221021200000F047FE00287F
:107DE000F3D0F6E7014B18607047C0469865FF1F57
:107DF00037B56B469D1D010004000222280003F0E8
:107E000063FE2B88B02B0ED12379122B09D12300CE
:107E1000FA331B78012B06D10121608800F0E0F8CD
:107E200001E01B2BF8D037BD10B5054B04211870AD
:107E300000F098F8FFF74CFDFEF770FB10BDC04650
:107E40009C65FF1F0020F0B50BB20F0087B0834286
:107E500034DA274B187803F0B7FC051E2BD00378D3
:107E6000A02B25D103AE3100FEF7E4F8041E0BD1A0
:107E7000B378DB0724D51F4B06341B68002B03D0D7
:107E80003100688898470400A868002801D003F0F2
:107E9000C3FC002C08D1184A039B1340174A934295
:107EA00006D0B3781B2B03D00121688800F098F826
:107EB000280003F0B1FE80200002784007B0F0BD3A
:107EC0000F4B1B68002B10D0310068889847041EA8
:107ED000DAD07378002BD7D1B27801A90A704B8021
:107EE0000C716888FDF7F6FFCEE70624F1E7C0467F
:107EF0009C65FF1F9465FF1F00FFFF00000112003B
:107F00009865FF1FF7B50190FC200D0017001E00BB
:107F100003F0EAFC04001320002C12D0B023200050
:107F20002370089BF4226770658026710830002B4F
:107F300008D0190003F018FC2100019803F094FD0B
:107F40000020FEBD089903F077FBF5E710B5041E8D
:107F500006D00078FD2803D803F0BEFCFF23237071
:107F600010BD00000A1F93B210B504000220032BBD
:107F700005D882400020024BD1529B189C7010BD46
:107F8000BC65FF1F0B8870B5043B04000D00022088
:107F9000032B0BD80121200000F04CFD030014201E
:107FA000002B03D02900200000F0DEFB70BD000094
:107FB00007B51300034A00920A00012100F02CFCCF
:107FC0000EBDC046ED81001107B50192032200925B
:107FD000024B0A00122100F049FC0EBD6B82001119
:107FE00007B56B4601AA11800449D880087806338A
:107FF000012802D1190003F0FFFC07BD9D65FF1F9A
:108000000C4B10B518700023FF210B4A138013810D
:1080100093819380094A53801370517293819372B4
:10802000D174D3821375517703F04EFC00F0FCF944
:1080300010BDC046CC65FF1FBC65FF1F9E65FF1FBE
:10804000F0B58DB06B46002003910C229B5E8342FD
:1080500000DBB0E05D4B187803F0B6FB051E00D1E5
:10806000A4E00378902B00D09DE006AF0100468885
:10807000380000F013FA79680400002900D19CE070
:108080003B88052B6ED13B89032B1CD905AC200006
:1080900000F0A2F86288172A61D83989131D994225
:1080A00031D17968237804310291D90738D56078C5
:1080B00000F08EF9071E06D0002303712378012BF0
:1080C00008D0132B23D0A868002800D178E003F053
:1080D000A3FB75E06288029909A800F0A6F8029057
:1080E000380000F08BF909AA2378387A019200222F
:1080F00031000092029A00F012F9380000F064F9A1
:10810000029B002BDFD0300000F080F9DBE7037822
:10811000032BD8D16288029909A800F0D6F8DEE7CF
:10812000122B13D1029909A800F0B5F8021EEAD16A
:1081300027498B88002BC6D0887909A9237801911B
:1081400061780091310000F0EAF8BCE7002302AA50
:1081500093833000617809AAFFF72AFFB3E71D4B2C
:108160000993F6E7042B02D09A1F012AABD8184ACC
:10817000043B9B00995A0029A5D0D2189078310071
:108180003A0000F0AEF800289DD13B88042B03D0C4
:1081900001213000FFF724FF012C04D1A86800283A
:1081A00001D003F039FB280003F036FD8020039B4B
:1081B0000002434018000DB0F0BD012800D182E755
:1081C00001213000FFF70CFFEDE7C046CC65FF1F33
:1081D000BC65FF1F010017000B7803704B784370DC
:1081E000CB788A781B021343438070470A880300C8
:1081F00002700A88120A42700A88012A06D14A8847
:1082000082704A88120AC27004207047022082429B
:10821000FBD14A8804309A704A88120ADA708A8838
:108220001A718A88120A5A71EFE710B5040001200A
:1082300082420CD94B780A781B0213432380834275
:1082400006D1CB788A781B0213436380002010BDCF
:10825000022BFBD1CB788A781B02134363804B79C6
:108260000A791B021343A380F0E70B8803700B8885
:108270001B0A43704B8883704B881B0AC3708B8822
:1082800003718B881B0A4371CB888371CB881B0ACF
:10829000C3710820704703000120082A14D14A78CE
:1082A0000878120202431A80CA78887812020243C0
:1082B0005A804A790879120202439A80CA798879E9
:1082C000120202430020DA80704710B5040001203A
:1082D000022A05D100204B780A781B021343238021
:1082E00010BDF8B5060010200F00150003F0FCFAD1
:1082F00004000120002C0ED0A0230C222900238092
:108300006780201D002D07D003F02EFA21003000D9
:1083100003F0AAFB0020F8BD03F08EF9F6E7F7B5ED
:108320001E00009008AB142017001D78019103F087
:10833000DBFA041E12D0A2230370019B4770438016
:10834000099B057146710C220830002B07D01900DB
:1083500003F00AFA2100009803F086FBF7BD0999A3
:1083600003F06AF9F6E737B5041E0FD04388002BF7
:108370000CD00025C1881323007A1722019500959F
:10838000FFF7CDFFFF2365806372257037BD0000C6
:1083900010B50C4904004A88002A09D08B89002BAB
:1083A00005D00020CB8A0222834201D010BD0122D9
:1083B00013000A20434300204032C854C8184280AA
:1083C0000472F3E79E65FF1F00234380037070472C
:1083D000094B00211A0010B55C88002C06D01C79CE
:1083E000844203D10A234B43D01810BD01310A3314
:1083F0000329F1D10020F8E79E65FF1F10B50400A6
:10840000407A03F069FAFF23637210BD70470430AD
:1084100010B580B203F068FB002803D00421494264
:1084200003F0DAFB10BD000070B50025104CA06809
:108430002580A581A580A84202D003F0EDF9A560B2
:1084400000250C4C0C4B606D1D80230058331D70B3
:10845000A84202D003F0E0F96565002560680028B5
:1084600001D003F0D9F9013508340A2DF6D170BDD9
:108470006466FF1F0866FF1F5866FF1F70B5041E65
:1084800009D1054D2880A881A880A868002802D0BD
:1084900003F0C2F9AC6070BD6466FF1FF0B54B8895
:1084A00085B00193002343600A7905000F00022A7A
:1084B00000D07BE0CA88032A17D98B685E781978C8
:1084C0003602DC78D8790E4399781B7A24021B0295
:1084D0000C43034353495BBA0B80331D93421ED1B7
:1084E000042C04D0631F022B0ED9012015E0019A41
:1084F0004D4B1201D35A002B06D00198FFF7BEFF57
:108500004A4A1369013313610421B8682E812C8013
:10851000494203F061FB6860002005B0F0BD434DA7
:10852000042C06D0631F022B0FD9EB680133EB60DC
:10853000DBE7019A3C4B1201D35A002B05D001987E
:10854000FFF79CFF2B6901332B61374B30000293FF
:10855000019B029A1B010193002301998C468B52C7
:10856000130063449C8003939E81FFF750FF039B9D
:10857000041E986016D00421B868494203F02CFB11
:10858000FA880100043A200003F0EEF80199029AFB
:10859000FB888A5A043B9B18029A8B522B68013342
:1085A0002B60A2E7AB690133AB619EE71E4B0293E0
:1085B000019B1E01029BF35A002B2DD002998C19AE
:1085C000A068002828D0012A26D1FA889B189BB2DF
:1085D0007352A189994217D39B1AC018B96803F046
:1085E000C3F8029BA289F35A934200D07DE7002290
:1085F0002B81A3882B80A3686B60029BF2520B4AED
:1086000053680133536070E7084A936801339360FD
:108610000198FFF733FF68E7044A53690133536158
:10862000F6E7C046CE65FF1F6466FF1FD465FF1FD7
:1086300070B5051E15D10B4C0B4B18802300583319
:108640001870606D002802D003F0E6F8656525001B
:1086500050356068002801D003F0DEF80834AC42E1
:10866000F7D170BD0866FF1F5866FF1FF0B51700F1
:10867000A12285B0920001934243394B06001B684A
:108680000C009B18D933FF331D78FDF741FF0430F0
:10869000854204DD3000FDF73BFF0430C5B2BD422A
:1086A00007D33A0000213000019B03F065F805B0C4
:1086B000F0BD2900380003F0EFF92300C6B25033B3
:1086C0001E700393019B29006365380003F094F842
:1086D000CBB20293002B02D0039B01361E70002602
:1086E0002300503303931B78B34204D8606D0028F5
:1086F00031D10020DBE7029A2800002A04D0013B98
:108700001000B34200D02800F700E719387003F0DA
:10871000FBF8786000280ED03A78019903F024F82D
:10872000019A3B780136D3180E4A0193D369F6B209
:108730000133D361D4E7039B18706065A74205D16C
:10874000084A1320D36A0133D362B0E7606803F0AC
:1087500063F80834F2E703F05FF800236365C8E7C5
:108760003409FF1FD465FF1FF7B50D000700042172
:10877000686803F031FA2B89040003702B891B0A07
:1087800043702B8883702B881B0AC3702E890225A7
:108790000436F6B2F42E15D81B4B9F4214D10C2090
:1087A00003F0A2F81135011E0CD0902303708E3B0C
:1087B0000371043B4380154B8460C680187803F036
:1087C00053F900252800FEBD5C237B43104AD318D3
:1087D0000093583301931B78002B0FD10300320014
:1087E00038000099FFF742FF019B05001B78002B22
:1087F000E8D13800009903F007F9E3E7054A0725B7
:10880000536A01335362DDE7FEFF0000CC65FF1FB2
:108810000866FF1FD465FF1FF0B587B000901720D2
:108820000F0016000193FFF7F2FD1325041E19D067
:108830000C98031E02D00199201D9847030AE3708B
:10884000052302AAA07004309081277000986670FA
:1088500003A993800494FFF787FF051E02D0200030
:1088600002F0DAFF280007B0F0BD0000F0B587B0D5
:108870001F000CAB1B780391059301210DAB060083
:108880001C78049200F0D6F81425002821D020008E
:10889000FFF77EFD0135041E1BD01149059B0A78A8
:1088A00003700132D2B2131EC68001D101231A0017
:1088B0000B7022713000049B03990097FFF7ACFF07
:1088C000051E09D1230021000648074A093302F09A
:1088D000D3FE280007B0F0BD002363802370F8E7C3
:1088E000D065FF1F6783001130750000F8B50500E3
:1088F0000E00064C064F2368002B02D031002800E2
:1089000098470434BC42F6D1F8BDC0467466FF1FD8
:108910008866FF1F0123064A5B42538000231371C0
:108920005362044A136053609360D36013617047CD
:108930008866FF1F7466FF1F0200002310B50649FA
:108940009C000859002801D1625010BD0133052B4D
:10895000F6D11320F9E7C0467466FF1F034A538817
:10896000181A434258414042104070478866FF1F22
:10897000F0B585B002930AAB1F780CAB1B88009052
:1089800008000E0001920393FFF7E8FF0500112095
:10899000002D1BD10E48FFF7E1FF04001520002C2D
:1089A00014D006220B99A771E01D02F0DDFE019B99
:1089B00030002371029B29006371009B6680237045
:1089C000039B6562E381FFF791FF280005B0F0BDCE
:1089D000FFFF000010B5FFF7C1FF04000220002CCC
:1089E00012D060880121FFF781FF606A002801D062
:1089F00003F0EAF828220021200002F01DFE0123E6
:108A000000205B426380207110BD000030B5074A32
:108A1000074C5588010013780020A54204D05B1A4A
:108A200059424B415842104030BDC0468866FF1F36
:108A3000FFFF0000084A10B501230C00904208D047
:108A4000FFF78CFF031E04D0037923405A1E934185
:108A5000DBB2180010BDC046FEFF0000024B1879C3
:108A6000431E9841C0B270478866FF1F70B504006E
:108A70000D001600FFF772FF002804D10D4B9C4239
:108A800000D0143070BD416A03790520002907D059
:108A900012221A40102A02D10520002EF2D10F20F6
:108AA000DB06EFD5897E0C20A94289414942494223
:108AB0000840E7E7FEFF0000030010B5002800D1E2
:108AC00010BD0348034A41889142F9D09847F7E71F
:108AD0008866FF1FFFFF0000002330B5C45CCD5C3B
:108AE0006C40D4540133102BF8D130BD0F23002239
:108AF00010B5C45C64002243CA54C25CD209013B75
:108B0000F7D210BD0200010010B52032103102F082
:108B1000D3FE10BDF0B58BB0039010200593170065
:108B2000049102F081FE0090102002F07DFE009B77
:108B300013240190002B05D000280CD11324009899
:108B400003F042F8019B002B02D0180003F03CF820
:108B500020000BB0F0BD102002F066FE06001020D1
:108B600002F062FE13240500002E00D1AEE00028C2
:108B700019D01022002102F05FFD32002900039875
:108B800002F09AFE041E0ED133787F2B51D83000AC
:108B90000099FFF7ABFF009B1B787F2B53D80199FF
:108BA0000098FFF7A3FF300003F00EF8002D02D06D
:108BB000280003F009F8002CC1D1102002F034FE87
:108BC0000600102002F030FE0290002E7CD000281B
:108BD00078D03A000F3223000125121105D00F334F
:108BE0003B4015B25A4253411BB26A1E1201002B80
:108BF00033D0049BD2B298180099029AFFF76CFF09
:108C0000013D10220021300002F016FDADB2049F9C
:108C10002D017D19AF4242D0002C33D0300002F03C
:108C2000D3FF029B002B00D189E7180002F0CCFF94
:108C300085E729003000FFF759FF28002549009AF1
:108C4000FFF74AFFA7E729000098FFF74FFF28002A
:108C50002049019AFFF740FFA5E70F210F40049933
:108C60008A18D9B28F4208D9D15C06A819540133A9
:108C7000102BF6D1029A0199C0E7791A4842414176
:108C8000C901F2E73900300006AAFFF725FF3200DC
:108C9000039806A902F010FE10370400BAE7002C72
:108CA000BCD13000029906AAFFF716FF320006A9D0
:108CB000039802F001FE082204003100059802F03A
:108CC00053FDABE71324A9E71324AAE7002800D03B
:108CD0006EE733E774BE0011F0B58BB00F001600DD
:108CE0000225009000283FD0002A3DD00B1DDBB2AA
:108CF0001800029302F098FD1135041E34D0FDF7E0
:108D000047FD05003A000099201D02F095FEEBB2E8
:108D10000393E3702B0CDBB22F0A00936370FFB256
:108D20002B0E2370A7700193FDF72CFD102201007C
:108D300006A802F081FE2100029A04AB06A8FFF704
:108D4000E9FE051E0DD1039B08223370009B04A988
:108D5000B370019B7770F370301D02F06DFEFDF76C
:108D60001DFD200002F030FF28000BB0F0BDF0B573
:108D70008FB00D00149E039004920593002A03D136
:108D8000022420000FB0F0BD002EF9D00398FFF7A9
:108D9000E5FD1424071EF4D07278337812021A43CA
:108DA000B3781B041343F27812061A43036A019244
:108DB000934201D30133E3D1002D03D03B79012449
:108DC0009B07DED50822002106A802F035FC059B92
:108DD00013240433DBB21800029302F025FD051EB4
:108DE000CFD0059A0499043002F026FE0422310007
:108DF000280002F021FE3900102210310AA802F0EA
:108E00001BFE2900029A06AB0AA8FFF783FE041E88
:108E10000FD1082206A908A802F00EFE0822311D73
:108E200008A802F0F9FD012807D101990398FDF780
:108E3000C9FC280002F0C8FEA3E70124F9E70000FE
:108E400070B51C4C05002368181E10D0002D14D1DD
:108E50001A78002A0CD1981C083202F085FC02F026
:108E600083FD0135002808D123681D70012070BDE5
:108E70000A331800082202F077FC2368002BF5D093
:108E8000122002F031FD061E0DD0C12321680370AF
:108E9000457002311022023002F066FC2368310076
:108EA000587802F0E1FD206802F08EFE0023236076
:108EB000DCE7C046B066FF1FF8B504002020FDF7D0
:108EC00055FB0D4EA700BB590500002B0DD0002807
:108ED0000BD0D878FF2809D108492A000C55F3593E
:108EE00007480333611802F0C7FBF8BD290002F000
:108EF000CBFB0028F0D1F8E7CC66FF1FB466FF1F5C
:108F000011A1001170B5064D84006359002B05D0E6
:108F1000D87802F0E1FCFF226359DA7070BDC046D8
:108F2000CC66FF1F70B506008CB00C001500002148
:108F30003022684602F080FB31001022684602F0C1
:108F40007BFD1D2021000322684402F075FD684668
:108F5000FFF7D8FD2D21040003222800694402F008
:108F60006BFD20000CB070BDF0B50700160097B087
:108F700001931CAB1D7830221EAB00910AA8002182
:108F80001C7802F059FB102239000AA802F054FDA7
:108F90001022002102A802F04FFB0722310002A894
:108FA00002F04AFD072202AB9818631E9C4101990A
:108FB00002F042FD02AB9C732B005A1E934102AAA1
:108FC000D3730021102206A802F036FB06221D9959
:108FD00007A802F031FD1A2002ABC01806221F9923
:108FE00002F02AFD102200990EA802F025FD1022A1
:108FF00002AB0EA908781C78013A6040D2B2087022
:1090000001330131002AF5D10AA8FFF77BFD1022B8
:1090100012A904000EA802F0A7FB102206AB0EA9AD
:1090200008781D78013A6840D2B2087001330131E6
:10903000002AF5D10AA8FFF765FD04431022209805
:10904000E4B212A902F0F8FC200017B0F0BD70B530
:109050000E0014008CB00100102268461D0002F0C2
:10906000EBFC3100082204A802F0E6FC21000822F3
:1090700006A802F0E1FC6846FFF744FD0400102258
:10908000280008A902F0D8FC20000CB070BDF8B58B
:1090900006000D0000243719AC4200D3F8BD02F0E1
:1090A00013FB030A3B70631CDBB201379D4203D9FB
:1090B0000234F054E4B2EEE71C00EDE773B50600AD
:1090C0000C000225002819D0002917D0032101A87F
:1090D000FFF7DDFF6B469A793F231A4001331343B4
:1090E0006A463000937101A92200FFF71BFF051E9D
:1090F00004D10322E01C01A902F036FB280076BD52
:1091000003785807DA08C00FD20080009B0710438D
:109110009B0F1843C0B2704707230B40C908C90012
:109120000B4303707047000070B50400FFF7EAFEC0
:10913000134DA4006359002B21D0186A002801D0D8
:1091400002F042FD2B59986E002801D002F03CFD40
:109150002B59D86E002801D002F036FD2B59186F1C
:10916000002801D002F030FD2B59586F002801D0A3
:1091700002F02AFD285902F027FD00232B5170BD73
:10918000CC66FF1F0E4B8000C35870B50C00002B3F
:109190000FD09D68002D0CD02B78201D0B706B78A4
:1091A0004B70A97CFFF7B8FF2B7E23726B69E360DD
:1091B00070BD10220021200002F03EFAF8E7C04600
:1091C000CC66FF1F014B18607047C046C866FF1F82
:1091D000074A03008000825810B5002A06D0D088C4
:1091E000984203D1012901D1FFF79EFF10BDC0466F
:1091F000CC66FF1FF0B5264E95B087000B93BB5988
:109200000500099112200A92002B31D0D888FFF76F
:10921000A5FB04001420002C2AD0280010A9FFF779
:10922000B1FFBB591E781D6A002E23D00895FDF7AB
:10923000EFFA07000020FDF7F1FA0790A379E61D89
:10924000069310AD0CA9089800F0E2FA0EA92800C8
:1092500000F0D7FA0B9B0A990493069B0998029396
:10926000079B0396019300970EAB0CAAFFF77CFEB9
:1092700015B0F0BDFDF7CCFA06903000FDF7CEFA40
:10928000E31DA779079310AB06000893DAE7C04601
:10929000CC66FF1F30B50C4C85002A59030085B001
:1092A0000120002A0ED018006946FFF76BFF2B59EA
:1092B0001A78D888054B002A00D1054B6A46072149
:1092C00000F0D9FB05B030BDCC66FF1F039800113C
:1092D0001198001130B5094C8500295985B010222C
:1092E0006846253102F040FA2A591121044BD088F2
:1092F0006A4600F0C0FB05B030BDC046CC66FF1F1B
:10930000AD98001130B5094C8500295985B010225F
:109310006846353102F028FA2A591121044BD088C9
:109320006A4600F0A8FB05B030BDC046CC66FF1F02
:10933000EB980011F7B54D4F86001020F4590D0041
:1093400002F072FAF3592062186A132200286CD0D6
:10935000033A29009C6802F007FAF3591A7801923F
:10936000002A58D11E6A227D317B94465140012249
:10937000019F114201D167461740217D9143394336
:109380002175377B4F40BC4660460027800701D4DB
:109390004F081740012102208F40227D82433A432B
:1093A0002275377B5740BC4660460027400701D4F2
:1093B00097080F400420227DBF0082433A43227564
:1093C000627D002794466046727B42400A4201D18A
:1093D00067460F400121627D8A433A436275777B7D
:1093E0005740BC4660460027800701D457080F400D
:1093F0000220627D7F00824317436775767B0022DF
:109400007E40760701D4BA080A400426617D9200A6
:10941000B1430A4362756A78002A08D06278002A4C
:1094200005D005220533DA7700221000FEBD0422A4
:109430002979114205D1A17C114202D10533033AA9
:10944000F1E7019A21782C78002A02D10A00210044
:10945000140018220429E8D8042CE6D8052060431B
:10946000034A05331218525CDDE7C046CC66FF1F85
:1094700084BE001110B50A001121024B00F0FBFA66
:1094800010BDC046479900110B0030B587B001AD43
:109490002B806B4604001100981D082202F064F92D
:1094A0002A000B212000024B00F0E5FA07B030BD86
:1094B0006F99001110B50A001121024B00F0DBFA80
:1094C00010BDC046C399001113B50B0011006A46C8
:1094D00013706B4604000622581C02F045F96A46D8
:1094E00008212000014B00F0C6FA13BDE3990011DA
:1094F00010B50A001121024B00F0BDFA10BDC046A4
:10950000339A00117FB505000B4BAA00D458080010
:10951000002C0FD0666F237FE28821780396266F98
:109520000296E66E0196A46E0094FDF709FC2800F1
:10953000FFF7FAFD7FBDC046CC66FF1F10B51721AF
:10954000FFF7E0FF10BD000070B50A000D00064BEC
:109550000221040000F08FFA060029782000FFF7AE
:10956000D1FF300070BDC0461399001170B586B0B0
:1095700000236A461370836804001D78681E0A2859
:1095800059D801A902F0E0FA060633373B3F4347BA
:109590004B4F5300180000F042F9062312284BD01D
:1095A00000281BD16088FFF7D9F90823002813D0C1
:1095B0004279002A47D1264B1A78072312070BD588
:1095C000244B1A680723002A06D01668002E03D001
:1095D000290001AAB04703006A4613706B461B7846
:1095E0006088002B2AD1FFF767FC06B070BD180019
:1095F00000F06CF9D4E7180000F087F9D0E7180004
:1096000000F093F9CCE7180000F0ADF9C8E71800B6
:1096100000F0C3F9C4E7180000F0F6F9C0E718003D
:1096200000F0F6F9BCE7180000F013FAB8E71800EC
:1096300000F013FAB4E707236A461370694660889E
:10964000FFF782FFD1E70523012AC5D1024BB8E716
:109650005965FF1FC466FF1FC866FF1FF8B52C4F72
:109660008600F35904000D00002B40D0DA888242B6
:109670003DD15A78062A33D11A78002A2ED00120FB
:1096800099681A6A097D014206D0157B054203D00C
:1096900007225A700120F8BD0220014204D0157B38
:1096A000054201D00922F4E70420014204D0127BD4
:1096B000024201D00B22ECE7164B1B68002BE9D0CD
:1096C0005B68002BE6D020009847BB5900215B78EF
:1096D000122BDFD12000FFF715FFDBE70E4BECE785
:1096E000112A04D1002900D032252900F2E7002DEB
:1096F00008D12000FFF732F9002803D010230279A7
:109700001343037121002800FDF798FAC2E7C04611
:10971000CC66FF1FC466FF1FC866FF1F70B50E4EE4
:109720008500AB590400002B13D01B78002B11D1FE
:109730000A4B1B68002B04D05B68002B01D0200073
:10974000984773595B78122B03D100212000FFF753
:10975000D9FE70BD024BECE7CC66FF1FC866FF1F49
:10976000C466FF1F094B8000C3581020002B0CD08B
:109770001A6A002A09D09B68002B06D0127A1B7E39
:10978000101C9A4200D9181CC0B27047CC66FF1F4B
:1097900070B503000D0014000220002A30D000290B
:1097A0002ED013700B78081D53704B789370FFF711
:1097B000A7FCE070012002212B7A23716B7B034010
:1097C00063716A7B0A401343042263716E7B164007
:1097D000334363716E7BF608F600334363712B7B72
:1097E0000340A371287B014000200B43A371297B18
:1097F0000A401343A3712A7BD208D2001343A371FA
:1098000070BD10B50A0001000120FFF7C1FF10BDB7
:1098100010B50A0001000220FFF7BAFF10BD70B5B5
:1098200006000C000220002E30D000292ED07378C4
:10983000201D0B70B3784B70F178FFF76DFC01229F
:109840003579257271794B10080013409340104010
:109850000343881010408000C9080343C9000B432C
:109860006373B1794B1008001340934010400343D9
:10987000881002409200C9081343C9000B432120FD
:109880002373FCF773FE854201D2122070BD2220A3
:10989000257AFCF76BFE8542F7D823781820042B35
:1098A000F4D86378012BF1D80020EFE7030010B55E
:1098B0000220002909D0002B07D00322481C0A707F
:1098C00019000D3201F050FF002010BD03000222EC
:1098D000080010B5002B06D0002904D00E32591C08
:1098E00001F042FF0022100010BD030010B502205D
:1098F000002909D0002B07D00422481C0A70190047
:109900000C3201F031FF002010BD10B5FFF7DEFF73
:1099100010BD03000220002906D0002B04D0052230
:1099200000200A701B784B70704703000220002B48
:1099300008D0002906D05B7800200B70013B082B73
:1099400000D918307047030010B50220002909D053
:10995000002B07D00622481C0A7019000A3201F0B9
:1099600003FF002010BD10B5FFF7B0FF10BD0200CF
:109970000B00022010B500290ED0002A0CD00721C0
:109980001970118859701188090A997011180822E4
:10999000D81C01F0E9FE002010BD03000A000220DF
:1099A00010B5002B0CD000290AD0997858780902FC
:1099B00001431180901CD91C082201F0D5FE002023
:1099C00010BD030010B50220002909D0002B07D0DC
:1099D0000822481C0A701900921801F0C5FE0020E8
:1099E00010BD02000B00022010B500290BD0002A88
:1099F00009D009211970117818185970511C0622C4
:109A000001F0B2FE002010BD10B5FFF75FFF10BDE2
:109A100002000B00022010B5002A09D0002907D04F
:109A20005178197011180622581C01F09DFE002073
:109A300010BD030010B50220002909D0002B07D06B
:109A40000A22481C0A701900063201F08DFE00201F
:109A500010BD10B5FFF73AFF10BD02000B00022049
:109A600010B5002A06D0002904D018005178FFF75D
:109A700053FB002010BDF0B585B017001E006A46EC
:109A800006230500080091819380FEF7C0FC132493
:109A9000011E02900CD03800B047041E05D12800EA
:109AA00001A9FEF76FFA041E02D0029801F0B4FE7D
:109AB0002800FFF701FA200005B0F0BDF0B5040062
:109AC0008BB0019115000021102202A801F0B4FD15
:109AD000334EA700B85900283CD0C388A34239D1DF
:109AE0000378002B36D14278062A18D102000100F3
:109AF000553235310C3006ABFFF7A9FA002829D1D1
:109B00002000FFF72FFE020006A902A801F02CFE9C
:109B1000200002A901F060FE01200BB0F0BD816EB3
:109B2000002917D00B8A112A28D19D420ED1019805
:109B30001231093A01F070FF012807D1BB5920000A
:109B40009D6EFFF70FFE29000200DEE732212000A4
:109B5000FFF7D8FC2000FEF701FF061E1BD0416A6C
:109B6000002918D00B8AAB4215D108220198123176
:109B700001F052FF01280ED1716A0AE09D42E9D13D
:109B800008220198123101F047FF0128E2D1BB59A8
:109B9000996E8A7EB9E7200001F01EFFBCE7C0463F
:109BA000CC66FF1FF0B56B4D87007E5985B03378CA
:109BB00002900393002B00D087E0B368346A0193CE
:109BC0007078062817D101221B7D134202D0217B19
:109BD000114218D10222134202D0217B114251D1ED
:109BE0000422134203D0237B134200D08BE0019B5D
:109BF0005A7DEB5991E007380428F8D801F0A4FF0A
:109C0000032E42678300B36E002B03D11C2001F0AA
:109C10000BFEB066EB599C6E002C1CD0102200216C
:109C2000200001F009FD0298FFF79CFD01002000D3
:109C3000FFF72DFA01F048FD2082200008211230A4
:109C4000FFF725FA0298FFF78DFDA076EB5921006A
:109C5000D888FFF70FFC0822EB591CE0B36E002BED
:109C600005D01A00198AF0881232FFF70DFC022283
:109C7000019B197DEB5911423DD0207B10423AD017
:109C8000073208E0F488FCF7DBFD01002000FFF755
:109C900011FC0A22EB595A70029B9C002A595378F6
:109CA000073B042B11D8D088FEF758FE00284ED071
:109CB000C3895A08D2182849029B0298CB542B59C1
:109CC00041180433254801F0D7FC05B0F0BDFCF77E
:109CD0009FFD03000120834201D100200393EB5933
:109CE000DE88FCF79BFD039902003000FFF7ECFBD8
:109CF000019AEB59117D042211420CD0217B1142B3
:109D000009D00B22C7E7F688FCF73CFD01003000C4
:109D1000FFF7EEFB6BE7019A527D01210A4204D066
:109D2000607B084201D00C22B5E702210A4204D030
:109D3000607B084201D00E22ADE704210A4204D024
:109D4000627B0A4201D01022A5E71222A3E7FA2281
:109D50005200B0E7CC66FF1FD066FF1F1BA10011A9
:109D600010B5064B1A780423100018401A4200D090
:109D70000348FFF727FA002010BDC0465965FF1FB2
:109D8000F043FF1F70B50400FFF7D4FA051E43D15E
:109D90002000FFF77FFA234EA400A0598268937C2D
:109DA000DB0708D50321036A1B790B40012B02D185
:109DB000017F0B430377431DD97F8B1E022B0DD8E8
:109DC000022900D00121C088FCF790FF04213359FB
:109DD0001A7F59700A431A77280070BD01290CD1E7
:109DE00002231022437000210C3001F025FC305971
:109DF00010213530FFF74BF9EEE70529ECD10223AE
:109E0000D118437010220C3001F0AEFC04233259FB
:109E1000117F0B431377EAE708251828DCD1053DAD
:109E2000DAE7C046CC66FF1FF0B58BB005914388DA
:109E30007E4F9E00F45915000493002C15D1012982
:109E400002D000200BB0F0BD101D57781678FFF738
:109E500057F9EB68320002932B7A04990193009032
:109E60003B002000FCF70CFFEBE7E388049A9342E9
:109E700001D00820E6E72378012B00D1D4E0059B30
:109E8000581E092800D9CFE001F05EFE05CE0A2950
:109E9000CC506C859AB229000498FFF773FFD1E784
:109EA000200029001022453001F05EFCB9594B78A2
:109EB000042B02D1013B4B70C3E70B000A00253392
:109EC00035320C310498FFF795F90498FFF702FA40
:109ED0000522431E9841BB59C0005A70B2E72000CA
:109EE00029001022553001F03FFC049B4F4C9D008F
:109EF000295904980A0006AB55320C31FFF77AF95C
:109F000029591022453106A801F086FD012808D103
:109F10000498FFF7F7F90590002804D106222B5981
:109F20005A7005988EE708230593FAE763780C2B9F
:109F30007AD1E36E002B03D11C2001F075FCE066A2
:109F4000BB59D86E00286FD01022290001F00CFCFC
:109F5000BB590498DC6EFFF705FC0D22A076BB59B7
:109F60005A706EE7E06E00285ED063780D2B5BD1EF
:109F70002B8808220382A91C123001F0F5FBBB5983
:109F80009A68517D0222114226D0186A407B104205
:109F900022D00C32E4E763780E2B45D1236F002BDF
:109FA00003D1162001F040FC2067BB59186F002830
:109FB00003D01022290001F0D7FB0F22BB59CFE7B5
:109FC00063780F2B30D1206F0622691C103001F00E
:109FD000CBFBBB599A68517D0422114203D0196A08
:109FE000497B1142D5D100210498FFF78BFA28E76D
:109FF000636F002B0DD0BB59586F0028F3D010228F
:10A00000290001F0B1FB0122BB5952425B6F1A617A
:10A01000E9E7142001F008FCBB5960675B6F002B77
:10A02000E9D126E72978DFE707200BE7CC66FF1F99
:10A0300010B5064C207001F087FB06212078FDF753
:10A0400091FF0348FEF778FC10BDC046DF66FF1F96
:10A05000D191001100200BB270B50D00834216DAC9
:10A06000264B187801F0B0FB041E0DD00378922B1C
:10A070000ED0A02B37D0224B1878FF283AD02100E1
:10A0800001F0F2FC002835D180200002684070BD4C
:10A0900043780E2B0BD03E2BEDD18378052B12D0BD
:10A0A000082BE8D181798088FFF7D8FA08E0154BB2
:10A0B00082889A42DFD183681878591CFEF7C0FE67
:10A0C000002817D1D7E7104B1B785B0712D50F4B31
:10A0D0001B68002B0ED09B68002B0BD0C289811D02
:10A0E00080889847ECE7FFF741FAA068002801D084
:10A0F00001F092FB200001F08FFDC5E7DF66FF1F36
:10A10000E943FF1F182000005965FF1FC866FF1FA5
:10A1100010B50078FFF712FA10BD10B50078FFF700
:10A12000FDFA10BD0C234343084A10B59B185A682A
:10A13000002A03D0012901D1904710BD9B68002B54
:10A14000FBD00029F9D19847F7E7C046FC66FF1F0E
:10A1500001238340094A10B5946B1C439463506BF0
:10A1600098435063D46B20009843012901D120000B
:10A170001843D063116B0B43136310BD0080004084
:10A18000F0B500240127154B85B0DA6B144E03920D
:10A190001A6C0192DA64019BE3403B4217D0039DA5
:10A1A000E5403D400295E5B202992800FFF7BAFF6D
:10A1B000316A736A002908D03900002B01D0029956
:10A1C00079402800FFF7C4FF01E0002BF9D10134EA
:10A1D0000C36172CDFD105B0F0BDC0460080004022
:10A1E000E066FF1F064B01215A68C2400A4204D0B4
:10A1F0001B68C3401800084070471B6DF9E7C04654
:10A20000008000400122064B8240002903D0D9681B
:10A210000A43DA607047D9689143D960FAE7C046CB
:10A220000038004030B5032444430F4BE25C1B1957
:10A230009C785D7801232D1B0135AB40013BA34089
:10A24000A140DB430C00122807D80849920052189D
:10A25000116819402143116030BD054A11680B4057
:10A2600023431360F8E7C046CBBE001108F000405E
:10A2700014F00040C21F70B5D4B20623092C0BD8CD
:10A280000125084C9540002908D00021FFF7CAFF9E
:10A2900023682B4323600023180070BD2368AB4361
:10A2A000F8E7C04600380040214BF0B51B185B783A
:10A2B000022B21D1032444431E4A1F4EA35C1219D2
:10A2C0009478012215008540B76B013CE4B23D4310
:10A2D000A240B563194C122815D89B0000290CD157
:10A2E00017495B1899680A439A600123205C154A54
:10A2F000834011680B431360F0BD11495B189968E6
:10A3000091439960F1E70E4B00290DD159690A4339
:10A310005A61225C1328E8D00123203A93400A496D
:10A32000086803430B60E7E7596991435961F0E717
:10A33000E066FF1FCBBE00110080004010BF00117F
:10A3400000F00040A0F00040A4F00040F8B5002468
:10A350001B4E1C4D1C4B1B5D012B1FD1194A9269D2
:10A36000E2401A420BD00122B25693402200143A26
:10A37000D2B2022A09D815494A6913434B61013404
:10A3800002360C35172CE5D1F8BD0022B2560F4924
:10A390009200521891680B439360F0E7022BEED1C4
:10A3A000E7B23800FFF71EFF01235840C1B2380062
:10A3B000FFF77AFF3800FFF715FF6877DFE7C04641
:10A3C0009DBE0011E066FF1FE166FF1F00F0004028
:10A3D000012202388240054B002903D059690A4303
:10A3E0005A617047596991435961FAE70038004052
:10A3F000F8B50E0001210F008740114A0400D36810
:10A40000FD43BB43D360831E8B4201D8FFF7E0FFBF
:10A4100000212000FFF72EFF0A4A0B4B5168012E46
:10A4200005D139431B1951605E700020F8BD2940E9
:10A43000516002221C1962709A6915409D61F4E70F
:10A440000038004000800040E066FF1F012210B588
:10A450008240074B002906D019680A431A6001217F
:10A46000FFF7C6FF10BD196891431960F7E7C046B2
:10A47000008000400C2370B5002543430A4A2900A0
:10A480009B181D70094B04001B185D70FFF7B0FF8F
:10A490000123A340064928000A681A430A600549B7
:10A4A0000A689A430A6070BDFC66FF1FE066FF1FE2
:10A4B000348000403080004070B504000E00FF285A
:10A4C00013D003250540FFF7D5FF084AA3089B00DA
:10A4D0009B183F22ED00AA40AE401968200091432E
:10A4E000314319600121FFF78DFE70BD183800401F
:10A4F000F8B50C244443134B0500E4186368002BA3
:10A5000003D1A3681220002B1AD0022201270E4B80
:10A5100000215B195A7028002770FFF769FF6368F4
:10A520001E1E08D0A3683E00002B04D02800FFF7B1
:10A5300059FE4640F6B228003100FFF709FE002020
:10A54000F8BDC046FC66FF1FE066FF1FF7B5C420DC
:10A55000FF222B4B80001958002491433F3A0A43B5
:10A560001A508022274F5202274E1A60274B1D5D3A
:10A57000002D21D0A31E012B03D80121E0B2FFF74B
:10A5800027FF012D18D11F4B9B69E3402B4213D0AD
:10A59000E3B218000193FFF725FE01000198FFF7D1
:10A5A00055FFE3B2143B022B1DD801217156184A06
:10A5B0008D405369AB4353613B7F002B0DD0E5B217
:10A5C0002800FFF795FF2800FFF70CFE7B7F0100B6
:10A5D000834202D02800FFF7A5FD01340C37023674
:10A5E000172CC3D1F7BD012100237156F3568D40BE
:10A5F000074A9B009B189A68AA439A60DCE7C0460A
:10A6000000E100E0E066FF1F9DBE0011E166FF1F54
:10A6100000F0004010B501210400FFF7E9FE01231E
:10A62000044A002011194B70A34091690B439361B8
:10A6300010BDC046E066FF1F70B50E001500040097
:10A64000FFF718FF0C236343094A20009B189D6005
:10A650005E60FFF74DFFF021064B074A8900051E9B
:10A660005A5002D02000FFF705FF280070BDC046F9
:10A67000FC66FF1F0000FF1F81A1001170B5134D84
:10A6800007202C78002C1FD198222100520028008E
:10A6900001F052F90123C420FF222B700C4B8000E3
:10A6A0001C635C630B4B1C605C600B4B1958914343
:10A6B0003F3A0A431A50802252021A600D20074A7C
:10A6C000074901F041F9200070BDC046E066FF1F58
:10A6D00000800040A0F0004000E100E04DA5001126
:10A6E0004DA30011030010B50620072B09D8054A19
:10A6F000137001F031FAD7210020034B034A89007F
:10A700005A5010BD1844FF1F0000FF1F8D1BFF1F74
:10A7100070B51D0002240C2910D8094ACA40D2077E
:10A720000CD5FBF72FFF041E08D1059A04992800C9
:10A73000FBF744FFFCF7B2FDFFF712FB200070BDF2
:10A740001210000030B50D7802232C009C431842F3
:10A7500001D02B431C0008252300AB43284201D025
:10A760002B00234320241D00A543204201D01C437D
:10A7700025002A230D70184204D011781E3B0B438C
:10A78000137030BD0028FCD10C2113788B43F7E700
:10A79000F8B51D0006AB1B88140007AA0E000B209D
:10A7A0001778002B27D10A78022A49D14A685078B5
:10A7B00011780002244A08438018042840D801F088
:10A7C000C3F903121D1B2300F06801F0DDF9021C20
:10A7D000C0B2B84200D93A1CD2B22000F1682A8037
:10A7E00000F0C2FF06E00222F3681B882A80237073
:10A7F0001B0A63700020F8BD0622EEE701232B80C0
:10A80000F3681B782370F5E7F368002B16D0082255
:10A810002A801A8822701A88120A62705A88A270D6
:10A820005A88120AE2709A8822719A88120A627112
:10A83000DA88A271DB881B0AE371DBE72B80D9E79A
:10A8400001202B80D7E7C04600D6FFFFF7B51600E2
:10A850000A781D0008AB1F880C000123022A18D1BA
:10A860004A685078117800022B4A08438018032860
:10A870000FD801F069F902254439E06801F084F944
:10A88000C0B20723B84204D37B190193152B02DD14
:10A890000D231800FEBDE0682A003100C01900F049
:10A8A00063FF6B4600209B88E268D0541B4B1B68FB
:10A8B000834203D01B68834200D098470023E8E717
:10A8C0000B23002FE5D1022DE2D1737832781B02E1
:10A8D0001343E2681380114B1B68002BEED01B68FA
:10A8E000002BEBD00120E8E70B23002FD1D1062D60
:10A8F000CED12A003100E06800F036FFDEE70B23FE
:10A90000002FC6D1012DC3D132787533012AC0D8AA
:10A91000E3681A70D2E7C04600D6FFFFEC68FF1F5D
:10A9200070B50C001500072837D801F00DF9041494
:10A9300036361B36242E182015290BD8184E162211
:10A940000021300000F078FE22002900300000F0E5
:10A950000BFF002070BD18200229FBD11288114B7B
:10A960001A80F6E718200829F4D10A000E482900B9
:10A9700001F0AAF8EDE718200129EBD10B4B107874
:10A980000B49DA69FFF7DEFEE3E718200129E1D180
:10A99000064B10780749DA6BF4E70220DAE7C04685
:10A9A000D468FF1F9644FF1F8C44FF1F1C44FF1FE9
:10A9B0004444FF1F6444FF1F030010B50020DB0761
:10A9C00004D50721024A034800F08CF810BDC046A8
:10A9D00028BF00111C44FF1F054A0300106800280F
:10A9E00003D082889A4201D1806870470068F6E7F8
:10A9F000E46AFF1F0A88030008009A4204D08A888C
:10AA000004309A4200D0002070470000F8B5F222CE
:10AA100000230D4F0D4E7968050042433370994273
:10AA200000D07B600A4C0021200000F005FE0023CE
:10AA30001A007C60AB4202D100203370F8BD0133B4
:10AA40002280DBB2F234F5E7DC6BFF1FDA6BFF1F0D
:10AA5000E86AFF1F73B56B46019006006846150053
:10AA60001980FCF74DFF041E11D1002D0FD07689FF
:10AA7000002E11D00C2000F0D7FE00280ED0084A7E
:10AA80000460136886808560002B02D1106020006E
:10AA900076BD1A001B68F7E70224F8E71324F6E7EF
:10AAA000E46AFF1F012100220A4B10B549420A4CFB
:10AAB000198099809A719A70084B20700120198032
:10AAC0005A60FFF7A3FF2078FCF778FF0448FDF7F2
:10AAD00033FF10BDF468FF1FE46BFF1FDC6BFF1F2B
:10AAE00091AB0011022310B5002802D0FFF7B2FF8E
:10AAF0000300180010BD0000030010B50020DB07A4
:10AB000004D50421024A0348FFF7A4FF10BDC04644
:10AB10003CBF00119C44FF1FF0B50E2687B0039385
:10AB20000CAB1F8802ABF61805000800310002923A
:10AB3000FDF768F804000120002C0FD03088FFF7E3
:10AB40004BFF03000E20002B08D05E68002E05D0BE
:10AB500021002800039B029A0097B04707B0F0BD80
:10AB60000A4B10B5984207D10122002352420A80B5
:10AB70008B708A808B7110BDFFF73CFF0028FAD0E4
:10AB800001235B42038000238370F4E7FFFF000092
:10AB9000F8B5050001290AD1134E00243388F227A5
:10ABA000AB4219D028001149FFF7DAFF06E002296D
:10ABB00004D10139FDF73EFF0028EDD0F8BD3B0080
:10ABC00063437268D018D35A002B09D03A00002191
:10ABD00000F032FD0134E4B2054B1B78A342EED8FD
:10ABE00001235B423380DDE7DC6BFF1FF468FF1F4E
:10ABF000DA6BFF1F10B5FFF7FDFE03000020834254
:10AC000000D0987810BD0000F0B589B01C000EABE4
:10AC100080CB03901E8810AB1B78049202930B7AB2
:10AC20000D00DB0616D42B780593022B24D0049854
:10AC3000FFF7D2FE002812D003689C46002B0ED0EE
:10AC4000029B2200019329003B0064460398009672
:10AC5000A04705E00498FFF7BFFE002802D10E20B0
:10AC600009B0F0BD8368002BF9D00A2229000398AF
:10AC700098470028D7D0F3E76B6858781A786B4B61
:10AC8000000210439842D2D8043B984210D2684B3D
:10AC9000984242D015D8674BC0180128C7D80B205E
:10ACA000002EDDD1EB681A7859683A80200028E040
:10ACB000614BC018032800D979E000F045FF846A91
:10ACC000789E5E4B9842B2D10B20002EC8D1012352
:10ACD0003B80EB6831001B7823706889013080B2BB
:10ACE000FCF790FF3A88031E0ED0017802328A18D2
:10ACF0003A80428962704289120AA27059680278C9
:10AD0000E01C00F031FD06E004323A8031000422FC
:10AD1000601C00F091FC0020A2E70B20002E9FD1C8
:10AD2000EB6807A91E8804233B80330A3000267095
:10AD30006370FCF767FF051E28D004AB9A890E23C9
:10AD400004A95B183E49C668FCF7D0FF00280BD168
:10AD50002B783C486A680599FBF786FB002803D1ED
:10AD6000012304AA5B42D3813278022A06D171689A
:10AD7000201D00F0F9FC3B8802333B800E2304AA1F
:10AD80009B181B88A3701B0AE370C4E704ABDE8129
:10AD9000F4E70B20002E00D062E7E9680398FFF784
:10ADA00029FF02233B802070000A6070B3E70B206C
:10ADB000002E00D054E70222EB681B883A802370F3
:10ADC0001B0A6370A7E7E86800F0DEFEC2B203006A
:10ADD0000720B24200D243E70DD00299DBB27118CE
:10ADE000994202DB921BD3B20293029BE9681A00DC
:10ADF0003B8089195AE70023F6E70B20002E00D08C
:10AE00002EE70722EB683A801A7822705A7862702F
:10AE10005A88A2705A88120AE2701A792271DA8866
:10AE20006271DB881B0AA37175E7C0460429000024
:10AE30000228000000D8FFFFFFD6FFFF0328000014
:10AE4000FFFF00006CBE0011F0B58DB06B46002016
:10AE5000089120229B5E83423DDAA64B187800F0D1
:10AE6000B3FC071E32D00378B02B2CD10079023806
:10AE700016281FD800F040FD17001E001E001E00FF
:10AE800031001E0096001E001D011E0052011E0012
:10AE900073011E00CD011E0050021E001E001E0088
:10AEA0008E021E00E302944B94491B8878880B8025
:10AEB000FBF71AF83800FCF79BFF914B1B68002B3F
:10AEC00001D038009847380000F0A6FE8020089B8B
:10AED0000002434018000DB0F0BDEE22002187486B
:10AEE00000F0AAFB0BAA3B7B7989388900923A00D3
:10AEF0000D32FCF79FFD0400804B1B78002C3FD1E6
:10AF000046E0804B788805937F4B4100CB5A0BAECF
:10AF1000073BDBB232880293002301937B4B210075
:10AF200006930093059BFFF76FFE744D002810D128
:10AF3000069B3A8A1B889A420BD138000599123039
:10AF400000F06AFD002804D02B7862899B00EB1882
:10AF50005A80162306A81B18328820007989FCF72E
:10AF6000C5FE2B7804009A00AA1851880029C3D086
:10AF70000133DBB22B70002807D006A9C98A918063
:10AF8000634A12889A42BCD802E00121494291806A
:10AF9000002B04D059497888FAF7DAFF8AE73E890E
:10AFA0000A2479E000253E89574B06937B88069A50
:10AFB0005B009B5A033B9D4202DB002DF0D05BE01F
:10AFC000162206A812183B7B798900923A003000BD
:10AFD0000D32FCF72FFD0590002858D04689017AE4
:10AFE0007888FCF7F1FC041E44D1464B788807931F
:10AFF000069B4100C95A454B0439C9B206AAD28AF8
:10B0000006930291019400930599079BFFF7FCFDBD
:10B01000041E2FD1069B39491A88931C002D26D176
:10B020004B807988384B4900CB5A5119033B8B42EE
:10B0300020DD059B31485B8941190B71A91C013545
:10B04000C9B2EDB2059145191B0A2B71059B2D491B
:10B050000433181800F088FB2C4B059A1B88D31872
:10B06000DDB22C4B9E4205D00136B6B29CE7498832
:10B070009942D6D0002D0CD0204C2800618800F0D9
:10B0800053FB207021007888FAF772FF12E7059CC5
:10B09000F0E7002C00D183E77B78142B00D109E77F
:10B0A00016493B794E800B700C717888FAF712FFC5
:10B0B00000E7162406ABE41821003889FCF7A2FD4E
:10B0C000011E00D1B7E1788822880F4C45002C5B27
:10B0D0000A4D013CE4B2029400240F4B0194009508
:10B0E000FFF792FD041E00D014E129007888FAF7DA
:10B0F0004FFFDFE6E46BFF1F8843FF1FFC68FF1F65
:10B10000F068FF1FF069FF1F2C65FF1FE06AFF1F3B
:10B110008643FF1FFFFF0000FE68FF1F162406ABDB
:10B12000E41821003889FCF76DFD011E00D182E191
:10B1300078882288AE4C45002C5BAE4D013CE4B2D1
:10B1400002947C89AC4B01940095FFF75DFD041ED1
:10B1500000D0DFE029007888FAF724FFAAE600256E
:10B16000A44B1D803B00F6331B78A24A78880792D7
:10B17000AB4208D99E4B12880693069943005B5A4E
:10B18000013B9A4203DB0799FAF716FF92E6162471
:10B190006B00FB18059306ABE418059B210018898A
:10B1A000FCF730FD011E03D1059B01241E8973E7C6
:10B1B0007888924B2288069C099343001B5B904E33
:10B1C000013BDBB20293002300960193099BFFF73A
:10B1D0001BFD041E02D0059B1E895DE77B88069A35
:10B1E0005B009B5A079A108832881218934202DC3F
:10B1F0001B1A013B33807F4C0230328809990019B9
:10B2000000F0B2FA2388328801359B182380EDB212
:10B21000A8E70BAA3B7B7989388900923A000D3266
:10B22000FCF708FC00250590059B002B04D10A249F
:10B23000002D00D16EE060E0059B7888197AFCF75C
:10B24000C3FB0100041E63D1694C6C4B78880694E3
:10B250000993069B4400E45A694B063CE4B20BAEEA
:10B26000328807930294019100930599099BFFF797
:10B27000CBFC041E4CD1079B5E491B881A1D002D78
:10B2800030D14A80059B5B4C5A8963191A716B1C3B
:10B290009BB2E318120A1A71162306A832881B18EB
:10B2A00079890598FCF722FDFF21AA1C2E1D033584
:10B2B0000B00059092B2B6B2ADB2002803D006AB37
:10B2C000DB8AD9B21B0AA218651911712B714C4D7A
:10B2D000301D2A884949201800F046FA2B88F618B4
:10B2E000B5B2A1E74988914207D17A880699520000
:10B2F000525AEB18053A9A42C4DC3E4C2800618849
:10B3000000F0CAFB207021007888FAF75FFED1E5D3
:10B31000002DF2D13E89BFE6162606ABF6183100A5
:10B320003889FCF76FFC3D000400FA3500282DD069
:10B33000037A9B060CD400227B8939897888009295
:10B340003A000C32FFF7E8FB041E10D03E8915E0EE
:10B350003088FFF741FB00281AD08368002B17D0F4
:10B360002100122278889847041EE4D0EEE72B785B
:10B37000002B02D17888FAF739FE00262B78002BB3
:10B3800000D097E5002C00D194E585E60124DDE7A7
:10B390000E24DBE7162506ABED1829003889FCF7EB
:10B3A00031FC041E47D0037A9B0611D4154A7B88D2
:10B3B0001188994203D01448814207D11380134B5E
:10B3C000F2261D780023D9B2A94221D30924A1E78E
:10B3D0002888FFF701FB00282FD08368002B2CD092
:10B3E0002100122278889847041EDFD092E7C046D9
:10B3F0002C65FF1FFC68FF1FFE68FF1FF069FF1F21
:10B40000E06AFF1FDC6BFF1FFFFF0000DA6BFF1F0E
:10B4100031005943546801336018615A0029D2D170
:10B420003C0008342100F22200F09EF921007888C7
:10B43000FAF7E4FD3EE501246CE70E246AE71D4BB4
:10B440001A887B889A4231D07888FAF7E1FD31E595
:10B45000F223059851684343CD18C95A00291FD0DB
:10B460003B7A012B0BD16C88AB887888AA1D00949D
:10B47000FFF752FB041E02D000233B722E88F222FB
:10B480000021280000F0D8F800232B80059B013311
:10B49000DBB20593084B05991B78064A8B42D7D837
:10B4A00001235B421380002CCED0F5E5002634004A
:10B4B0000596EFE7DC6BFF1FDA6BFF1F70B504002A
:10B4C0000E001500FFF796FA031E08D1310005485B
:10B4D000FFF790FA03001120002B02D01C800020FF
:10B4E0009D7070BDFFFF0000F8B50B4F06003B7864
:10B4F0000D001400FF2B0ED00A2000F0F5F9011EFC
:10B5000009D0B1230380002346800371C5800481E4
:10B51000387800F0A9FAF8BDDD44FF1FF7B50F0039
:10B5200008A90600088809A90B240988002821D148
:10B530000234022B1ED1557813782D021D432B00A7
:10B540008B4301937334002B14D1FB683000190036
:10B550000093FFF74FFB019C85420BD02A0030007F
:10B560000099FFF7ABFF041E04D12A00300079894F
:10B57000FFF7BAFF2000FEBDF0B50E7885B003904E
:10B580000AA805880120022E0DD14C68277864781E
:10B5900024023C43054FBC4205D10398DBB201961F
:10B5A0000095FFF7BBFF05B0F0BDC04602290000C3
:10B5B000034B10B51B68002B00D09847FEE7C04630
:10B5C000E86BFF1F07B501A8FFF7F2FF044A054823
:10B5D0000021121A00F0B0F9F8F70CF9FEE7C046A6
:10B5E000EC6BFF1FE044FF1F01B40248844601BC1E
:10B5F000604700BF5136FF1F01B40248844601BCBA
:10B60000604700BF4550000001B40248844601BCB9
:10B61000604700BF3D18000001B40248844601BCE9
:10B62000604700BFCD3BFF1F01B40248844601BC08
:10B63000604700BFB532FF1F01B40248844601BC19
:10B64000604700BF154D010001B40248844601BCAB
:10B65000604700BFEDA5000001B40248844601BC6C
:10B66000604700BF456B010001B40248844601BC3D
:10B67000604700BF8552010001B40248844601BC06
:10B68000604700BFA946010001B40248844601BCDE
:10B69000604700BF5147010001B40248844601BC25
:10B6A000604700BF7536FF1F01B40248844601BCE5
:10B6B000604700BF3555000001B40248844601BC14
:10B6C000604700BF5952010001B40248844601BCE2
:10B6D000604700BF2951010001B40248844601BC03
:10B6E000604700BF253AFF1F01B40248844601BCF1
:10B6F000604700BFC51D000001B40248844601BC7C
:10B70000604700BF4D1F000001B40248844601BCE1
:10B71000604700BFDD32FF1F01B40248844601BC10
:10B72000604700BFF94C010001B40248844601BCE7
:10B73000604700BF350E000001B40248844601BCDA
:10B74000604700BFDD66010001B40248844601BCC9
:10B75000604700BFC926000001B40248844601BC0E
:10B76000604700BFC521000001B40248844601BC07
:10B77000604700BFE94C010001B40248844601BCA7
:10B78000604700BF0519FF1F01B40248844601BC91
:10B79000604700BF75A9000001B40248844601BC9F
:10B7A000604700BF156B010001B40248844601BC2C
:10B7B000604700BF8B52010001B40248844601BCBF
:10B7C000604700BFC94A010001B40248844601BC79
:10B7D000604700BFF54E010001B40248844601BC39
:10B7E000604700BF311B000001B40248844601BC21
:10B7F000604700BF8D30FF1F01B40248844601BC82
:10B80000604700BF090E000001B40248844601BC35
:10B81000604700BFB939FF1F01B40248844601BC2C
:10B82000604700BFD949010001B40248844601BC09
:10B83000604700BF3D4B010001B40248844601BC93
:10B84000604700BF0124000001B40248844601BCE7
:10B85000604700BFC9A9000001B40248844601BC8A
:10B86000604700BF5D17000001B40248844601BC78
:10B87000604700BFED4A010001B40248844601BCA4
:10B88000604700BF7530FF1F01B40248844601BC09
:10B89000604700BF2D2EFF1F01B40248844601BC43
:10B8A000604700BFA13AFF1F01B40248844601BCB3
:10B8B000604700BF1D4B010001B40248844601BC33
:10B8C000604700BFE548000001B40248844601BC5F
:10B8D000604700BF7918000001B40248844601BCEB
:10B8E000604700BF1147010001B40248844601BC13
:10B8F000604700BF1D4D010001B40248844601BCF1
:10B90000604700BFF53BFF1F01B40248844601BCFD
:10B91000604700BF017F000001B40248844601BCBB
:10B92000604700BFB54C010001B40248844601BC29
:10B93000604700BF2526000001B40248844601BCD0
:10B94000604700BFB70E000001B40248844601BC46
:10B95000604700BF1531FF1F01B40248844601BC97
:10B96000604700BFF30E000001B40248844601BCEA
:10B97000604700BFD91B000001B40248844601BCE7
:10B98000604700BF6571010001B40248844601BCF4
:10B99000604700BF056A000001B40248844601BC4C
:10B9A000604700BF0139FF1F01B40248844601BC53
:10B9B000604700BF8D12000001B40248844601BCFC
:10B9C000604700BF0D52010001B40248844601BC2B
:10B9D000604700BFF937FF1F01B40248844601BC2D
:10B9E000604700BF091B000001B40248844601BC47
:10B9F000604700BFA54F010001B40248844601BC66
:10BA0000604700BFE117000001B40248844601BC52
:10BA1000604700BF3119FF1F01B40248844601BCD2
:10BA2000604700BFCD4C010001B40248844601BC10
:10BA3000604700BF792EFF1F01B40248844601BC55
:10BA4000604700BF4551010001B40248844601BC73
:10BA5000604700BF0D34FF1F01B40248844601BC9B
:10BA6000604700BF6DBC000001B40248844601BCC1
:10BA7000604700BF594F010001B40248844601BC31
:10BA8000604700BF055E000001B40248844601BC67
:10BA9000604700BF291C000001B40248844601BC75
:10BAA000604700BF090E000001B40248844601BC93
:10BAB000604700BF350E000001B40248844601BC57
:10BAC000604700BF691F000001B40248844601BC02
:10BAD000604700BF810E000001B40248844601BCEB
:10BAE000604700BF5522000001B40248844601BCF3
:10BAF000604700BFE928000001B40248844601BC49
:10BB0000604700BFC56D010001B40248844601BC16
:10BB1000604700BF9DA9000001B40248844601BCF3
:10BB2000604700BF2146010001B40248844601BCC1
:10BB3000604700BF851F000001B40248844601BC75
:10BB4000604700BF4537FF1F01B40248844601BC6F
:10BB5000604700BFE13BFF1F01B40248844601BCBF
:10BB6000604700BF8D1BFF1F01B40248844601BC23
:10BB7000604700BF4536FF1F01B40248844601BC40
:10BB8000604700BF2124000001B40248844601BC84
:10BB9000604700BFDD52010001B40248844601BC89
:10BBA000604700BF3939FF1F01B40248844601BC19
:10BBB000604700BFADAE000001B40248844601BC3E
:10BBC000604700BFB352010001B40248844601BC83
:10BBD000604700BF014C010001B40248844601BC2B
:10BBE000604700BF5549010001B40248844601BCCA
:10BBF000604700BFB14E000001B40248844601BC5A
:10BC0000604700BF5125000001B40248844601BCD2
:10BC1000604700BF7939FF1F01B40248844601BC68
:10BC2000604700BF434D010001B40248844601BC97
:10BC3000604700BFED38FF1F01B40248844601BCD5
:08BC4000604700BFCD3AFF1F71
:10BC480000010103020203030403050206020702BE
:10BC5800080209030A030B030C020D000E030F036D
:10BC6800100311031303140315001600A53B00115C
:10BC7800D93B001100000000020000008ABC00113E
:10BC8800192A0F180A000000F1590000FD240000CD
:10BC9800414601004180001155A00011A97400110E
:10BCA800457E00112D53001149AE0011794F001146
:10BCB800B53D0011E53E0011000000001616000019
:10BCC80002000000D4BC0011F4FFF3FFD2FC000016
:10BCD8002540001100000000000000005475796143
:10BCE8000042312E34003030313500676974687590
:10BCF800622E636F6D2F7076767800544830350069
:10BD0800020000001CBD0011292A282A272A262AF9
:10BD1800252A242A0A180000E20400007102000003
:10BD280078EC0000744000001027000060F000006C
:10BD380006640000204E000000000000050000001E
:10BD48001F501D00023CB400000115001400000043
:10BD5800A1020000303132333435363738394142A8
:10BD68004344454600000000315700118557001133
:10BD7800000000000200000088BD00116F2A6E2A32
:10BD88001A18EAD8BC80F0FC60000000000000002F
:10BD98000000F303B59747D6F613F7D777E6F0A771
:10BDA800F474000001A00000000000006410B71D3A
:10BDB800C8206E3BAC30D9269041DC76F4516B6BD1
:10BDC8005861B24D3C7105502083B8ED44930FF093
:10BDD800E8A3D6D68CB361CBB0C2649BD4D2D38649
:10BDE80078E20AA01CF2BDBDFB349B5F8000008096
:10BDF8000010000000000000AB6000113577001152
:10BE0800CF6000113D7B001153610011137B0011BD
:10BE1800C9610011E97A00111B620011B17C00119F
:10BE280083620011B17C0011B56200116B7C0011B6
:10BE3800C9610011A17A001141620011497C001109
:10BE4800000000000000000027630011497C001179
:10BE5800896300114D770011052A042A012A002A56
:10BE680002290328012800280118001800000000F2
:10BE7800000000000000000000000087010102012E
:10BE8800020101020102030304010301010101018E
:10BE98000303020103000D000E001000110013003F
:10BEA8001401070108010A010B011C011D0204020B
:10BEB80005020702080219021A021C021D030103E7
:10BEC800020317000201000504000807000B0A001E
:10BED8001716001D1C010201010504010E0D0111B8
:10BEE80010011413011716011A19020201020B0A94
:10BEF800020E0D0211100214130217160305040393
:10BF08000807030B0A030E0D0001020307090A0BB9
:10BF18000E0F101112141718191A1B1F20212200B6
:10BF280091A700114DA800110000000002000000B8
:10BF380072BE00110000000079B500110000000079
:08BF48000200000070BE0011B0
:020000041FFFDC
:10000000000000001D3D001190BC00118CBC0011CF
:100010001062FF1F00000000000000000000000050
:1000200000000000000000000000000000000000D0
:1000300000000000000000000000000000000000C0
:1000400000000000000000000000000000000000B0
:1000500000000000000000000000000000000000A0
:100060000000000000000000000000000000000090
:100070000000000000000000000000000000000080
:100080000000000000000000000000000000000070
:100090000000000000000000000000000000000060
:1000A0000000000000000000000000000000000050
:1000B0000000000000000000000000000000000040
:1000C0000000000000000000000000000000000030
:1000D0000000000000000000000000000000000020
:1000E0000000000000000000000000000000000010
:1000F0000000000000000000000000000000000000
:1001000000000000000000000000000000000000EF
:1001100000000000000000000000000000000000DF
:1001200000000000000000000000000000000000CF
:1001300000000000000000000000000000000000BF
:1001400000000000000000000000000000000000AF
:10015000000000000000000000000000000000009F
:10016000000000000000000000000000000000008F
:10017000000000000000000000000000000000007F
:10018000000000000000000000000000000000006F
:100190000133FF1F6131FF1FC16601000000000035
:1001A000000000000000000000000000000000004F
:1001B000000000000000000000000000000000003F
:1001C000000000000000000000000000000000002F
:1001D000000000000000000000000000000000001F
:1001E000000000000000000000000000000000000F
:1001F00000000000000000000000000000000000FF
:1002000000000000000000000000000000000000EE
:1002100000000000000000000000000000000000DE
:1002200000000000000000000000000000000000CE
:1002300000000000000000000000000000000000BE
:1002400000000000000000000000000000000000AE
:10025000000000000000000000000000000000009E
:10026000000000000000000000000000000000008E
:10027000000000000000000000000000000000007E
:10028000000000000000000000000000000000006E
:10029000000000000000000000000000000000005E
:1002A000000000000000000000000000000000004E
:1002B000000000000000000000000000000000003E
:1002C000000000000000000000000000000000002E
:1002D000000000000000000000000000000000001E
:1002E000000000000000000000000000000000000E
:1002F00000000000000000000000000000000000FE
:1003000000000000000000000000000000000000ED
:1003100000000000000000000000000000000000DD
:1003200000000000000000000000000000000000CD
:1003300000000000000000000000000000000000BD
:1003400000000000000000000000000000000000AD
:10035000000000000000000000000000000000009D
:10036000000000000000000000000000000000008D
:10037000C5B50011000000000000000000000000F2
:10038000000000000000000000000000000000006D
:10039000000000000000000000000000000000005D
:1003A0000000000000000000000000000D1BFF1F07
:1003B000000000000000000000000000000000003D
:1003C000000000000000000000000000000000002D
:1003D000000000000000000000000000000000001D
:1003E000000000000000000000000000000000000D
:1003F00000000000000000000000000000000000FD
:08183800F06FFF1F4118FF1FB4
:10184000024981F3088802F0A7FB0000F06FFF1F38
:1018500070B500241E491F4A1F484C6308CA1B0567
:101860001B0DE4188242F9D11C4B80228B630021AE
:1018700009201B4B920519621A4B1B4DDA671B4B53
:10188000DA688243DA609A68194802409A60112047
:10189000296002F091F8112002F06EF880226B6C42
:1018A000112093436B64EE23DB006343114A1B0C4E
:1018B00013840122104B9A7201F008FC0F4B1B7825
:1018C000002B04D10E4B1021187802F0FDFB70BDE7
:1018D000000005408805054000060540FF010000A6
:1018E00000F0004004E100E0003800403CF000401F
:1018F000FFDFFFFFE061FF1F9462FF1FC264FF1F55
:10190000C062FF1F10B502F0AFF9072804D01228FB
:1019100008D0022808D010BD044A0420136B0133FC
:101920001363F8E70220F6E71420F4E7D465FF1FFD
:10193000F8B507000C0026002500503630785135E8
:10194000002804D10300287058342370F8BD29788A
:10195000CA00481E8141A3183800A25C5B68C9B266
:10196000FFF7D0FF00280DD12B78DA00A218013341
:1019700050602B703378044A013B3370136A013393
:101980001362D8E70123DFE7D465FF1F5C234343DD
:10199000074910B5C9180B0058331B78012B05D126
:1019A000FFF7C6FF034A936A0133936210BDC04636
:1019B0000866FF1FD465FF1F10B502F0C5FA064A7E
:1019C0000121130010CB4942D967044B136002F088
:1019D0009BFB200010BDC04600E100E0100010009D
:1019E00010B5040002F0B0FA024B1C6002F08CFB50
:1019F00010BDC04600E100E0431E5A425341A02200
:101A0000F0B5D2015B421340154D164A40019B18B8
:101A10002A18127E8BB00191002A1BD01A000832BE
:101A2000D46F0022E6B206AFE4B294420EDC28186E
:101A3000C369002B08D0019902AA117106AA049269
:101A400002AA167303A898470BB0F0BD1978B954D1
:101A50000132EAE71A7D1A7806AB01261A70E6E72A
:101A60009468FF1F00400040F0B5254B0400400182
:101A7000C25C85B0002A2BD01A18117E002927D00D
:101A8000917E002924D01179022921D11689D78885
:101A9000D168F51BADB22A1C102D00D9102292B2CC
:101AA000BE4217D11818012303710023C269C380F5
:101AB00003819A4206D068460321037301710293A1
:101AC00001A890470820002C00D0192001F0FEFA50
:101AD00005B0F0BD013C65426C41A0256442ED01BA
:101AE0002C40084D1B186419074D0633013A92B279
:101AF000AA42EDD01888461C1E80085C2070F5E7CD
:101B00009468FF1F00400040FFFF00000F220E4BB3
:101B100010B59868104002380A280BD802F060F817
:101B20000D0A0B0A0A110A0A0A0A060002210020FD
:101B3000FFF762FF10BD0121F9E70020FFF794FFD6
:101B4000F8E7DB6FF6E7C046004000400F220E4B7F
:101B500010B59868104002380A280BD802F040F8F7
:101B60000E0A0B0A0A120A0A0A0A060002210120BA
:101B7000FFF742FF10BD01210800F9E70120FFF740
:101B800073FFF7E7DB6FF5E70090004013B5334CC8
:101B90002378072B3DD8324B1A78324B002A39D1A3
:101BA0008022196852020A431A60252001F0C4FEFF
:101BB00020232D4A11680B43802113606B460422B9
:101BC000C90508680733104228D080210422C905BE
:101BD000C86810422ED080212020C905CA688243DF
:101BE000CA6014221A701A78002A2FD18021C905E0
:101BF000C86820320243CA6014221A701A78002A78
:101C000028D11A4B1A7D22785A601D221A70593237
:101C1000DA6013BD1A6816490A40C5E7086802432E
:101C20000A6014221A701A78002ACED01A78013A63
:101C3000D2B2F7E7C8680243CA6014221A70197852
:101C40004A1ED2B21A700029F9D1C4E71A78013AB3
:101C5000D2B2C7E71A78013AD2B2CEE71844FF1FD2
:101C6000E044FF1F3CF000401044FF1F00200040F4
:101C7000FFFFFEFF564B70B51B68012B03D1554A81
:101C8000936D0133936502F0CFF9534B534A1860BB
:101C9000534B544C1A600123534A1360534A136048
:101CA0002378002B06D006225149524802F0DCF876
:101CB00000232370504A514B10681B78C1B2002B8F
:101CC0000ED14F4CC0B223785BB2002B4FDB237890
:101CD00024785BB264B21B0424021B191B18136026
:101CE0000B1C50294ED95023464A47491078DBB285
:101CF000FF2202284BD10868444C454D267890437A
:101D00002A78964254D9227824782E78023B5D10A6
:101D1000A31B6B435201D31A10335B1118430860A5
:101D200002F092F8031F012B45D83A4B1B78002B89
:101D300006D0394B1B78002B02D0002002F034F97A
:101D4000A122364B92009978354B4A431B689B1869
:101D5000832292009B181B78033B012B03D8AF20F2
:101D6000400001F0F9FF01222E4BDA8270BD23788A
:101D700024785BB264B2FF33FF341B0424021B19C6
:101D80000138ABE7CAB2022AAED20223ACE7086838
:101D9000254C264D267890432A78964208D92278F9
:101DA00024782D78023B5B10641B63435201B2E739
:101DB0002378DBB2B2E70228D5D11D4B1B78013B5B
:101DC000022B03D91B4B1B78022BCCD16C20C8E70C
:101DD0009809FF1FFC0FFF1F0C65FF1FFF3F00004E
:101DE000141003401065FF1F0C1003400010034047
:101DF000D50BFF1F7211FF1FB40003408C09FF1F9A
:101E0000680AFF1F490AFF1F94000340460AFF1F8C
:101E1000470AFF1FF908FF1F2209FF1F300DFF1F90
:101E20003409FF1FBC0BFF1F440AFF1F450AFF1F99
:101E30001C09FF1F2309FF1F10B502F015F900222E
:101E4000014B1A8010BDC0460865FF1F10B502F097
:101E500043F8A121054A89009478054A6143126834
:101E6000044B5218528C1A8010BDC046300DFF1F13
:101E70003409FF1F0865FF1F10B50D4B0D4A9978F7
:101E8000A1239B004B431268D218531DD97F0A4BE4
:101E90001B88994209D2441C07D0C82805D0D269B2
:101EA0005B1A5A43054B5343C01802F015F910BD95
:101EB000300DFF1F3409FF1F0865FF1F710200006E
:101EC00070B5244D2B68002B28D002F0F5F82B6854
:101ED000D8402B680400002B27D002F06DF82B6847
:101EE000D8401D4B1D4A9978A1239B004B43126893
:101EF000D118D25C91239B00002A20D0CA5801320D
:101F0000CA50174B17491B680868834214D3D23B49
:101F1000181A012A1AD0144B186070BD02F0CCF8C0
:101F2000124B196801F070FFD3E702F045F80F4B30
:101F3000196801F069FFD4E70D495B18E8E7CA505A
:101F40000C4B1B68DB68E418201AE4E7F530FF301F
:101F5000E1E7C0461C08FF1F300DFF1F3409FF1FBB
:101F60009C09FF1F0C65FF1FA009FF1F1808FF1F1A
:101F70002DFF3F001465FF1F70B504000D002829D8
:101F800016D10300A433C2881B889B1A0B4A9BB24C
:101F900093420DD906006A3605223100653001F002
:101FA0003BFE002804D13100200002F07DF870BD16
:101FB0002900200001F008FFF9E7C046FE7F00007D
:101FC000F8B50500012001F0B7FF134CA36AA26A1F
:101FD0009342FBD1114E336002F016F81049030012
:101FE00008601048426894460F4A17680022BC45B2
:101FF00001D24268BA1A0D4802603268AD18A422B4
:10200000E562606A520302436262094A1278002A5A
:1020100001D00F3B0B60F8BD00F00040340AFF1FF9
:10202000E408FF1F28100040180AFF1F1C0AFF1FAA
:102030001C09FF1F70B580241025E405A3682B43FD
:10204000A36001F059FEA368AB43A36070BD00001C
:10205000F7B5160080221C001023D205019191686B
:1020600005000B43936000225A4BD7301A6001F0F1
:1020700043FF9D232A002F009B00EB58CA32012109
:102080000092FC37002B01D00021009A386801F043
:10209000B3FF2900009BCB311A784F4BD3351A6020
:1020A0004B780A781B0213438A7812041A43CB78C0
:1020B0001B061343494A1BBA13604B790A791B026A
:1020C00013438A7912041A43CB7931001B06134358
:1020D000434A1BBA13606B782A781B021343AA7811
:1020E00012041A43EB781B0613433E4A1BBA1360D3
:1020F000019A330213433C4A13603C4B22001B1BE2
:102100009C4603293DDCB3089A0013005142B21AE1
:10211000032A46D1354AE018511A827840781204D1
:1021200000020243E05C043302430A600022FF2BFA
:102130004BDDF0222E4B12011A600F222D4B1A603C
:102140002D4A1368002BFCD00023224A2749136034
:10215000091B321D0B191B68043A180A23706070A2
:10216000180C1B0EA070E3700434002AF2DC8022ED
:1021700010213B68D20501333B6093688B43936029
:10218000F7BD6346D578981893782D061B042B432A
:10219000157804392B43557804322D022B43036004
:1021A000AFE7022A0AD1114AE05C511AE2185278CC
:1021B000120202430A6004339BB2B7E7012AB5D189
:1021C0000A4A521AE15C1160F5E7084959180A6099
:1021D0000433ACE7000004403C00044038000440F5
:1021E00034000440300004400C000440000104406E
:1021F000040004401000044014000440F7B515002A
:1022000080221C001023D2050091916807000B4327
:1022100093600023654AD730136001F06DFE9D2363
:102220003E009B00F9583B00CA363200FC330029BF
:1022300000D07FE0586801F0DFFE390032785C4B57
:10224000CB311A604B780A781B0213438A78AC466C
:1022500012041A43CB78281D1B061343554A1BBA98
:1022600013604B790A791B0213438A7912041A43CB
:10227000CB791B061343504A1BBA13604B7A0A7A78
:102280001B0213438A7A12041A43CB7A21001B06DD
:1022900013434A4A1BBA1360009A2B021343484A5D
:1022A00013602200474B1B1B0093009BCE785B18EA
:1022B00001938B7836061B0433430E78043833437E
:1022C0004E78043136023343019E33600328ECDC40
:1022D0000321A808431C9B002940800003292BD11F
:1022E0003849E5185E18A9786D78E35C09042D0279
:1022F000294319433160030008330021FF2B2DDDF2
:10230000314B324919600F21314B196001232749A4
:102310000B60304B19680029FCD006211B680B406C
:10232000042B20D080220020D20593680A318B43F1
:102330009360FEBD01217DE7022908D121495D1886
:10234000E1184978E35C090219432960D3E70129C0
:10235000D3D11C495918E35C0B60CCE71948181815
:1023600001600433CAE7002310490B606346002B69
:102370000CDC3B00FC335A68102101325A60802289
:10238000D205936801208B439360D2E7009B9B1892
:102390001B68190A13705170190C1B0ED37004239B
:1023A0005B4291709C440432E0E7C0460000044068
:1023B0003C00044038000440340004403000044035
:1023C0000C0004400001044004000440080F000019
:1023D000100004401400044070B5061E19D00222FB
:1023E0005A4B9B799343012B13D1594B1A78FF2AEF
:1023F0000FD15A78FF2A0CD19A78FF2A09D1DA78BE
:10240000FF2A06D11A79FF2A03D15B79FF2B00D16D
:1024100099E0504B0C201A78012A08D000224E4D2A
:102420001A7029780B00093B042B01D8212070BDBC
:102430004B1F012BFAD9454CA37B042B00D982E01A
:10244000A279032A00D97EE09A1ED2B2012A02D8CC
:1024500060881F2877D9002E56D0012E73D1A0880E
:102460000128E3D0002907D1581E032803D801F022
:10247000B7FB121715122E702978481E032811D8A1
:102480000025364B1D602823237501F095FCA842DA
:1024900027D0A580CAE702212970EDE70421FBE7D8
:1024A0000321F9E707390129C0D82D490968C96A0C
:1024B0008906BBD52B4908780028B7D1012A01D954
:1024C000002BB3D102230B708021274D26338901C5
:1024D0002878237501F000FC80212878890101F01B
:1024E000F3FD0123A380214B1B78002B0AD0FA2295
:1024F00080211F4B92001B8809025A431A4B1878FF
:1025000001F0A2FB002092E701F01EFD2B78A680CF
:10251000073B012B03D917482E7001F09DFC114B8E
:10252000114C1A78002A06D08021002220788901D7
:102530001A7001F0D1FB01F0E7FD8021207809023B
:1025400001F0CAFBDEE7122071E7C046A60BFF1FB1
:102550006B09FF1F1A09FF1F1C09FF1F4809FF1FF6
:102560001465FF1F2309FF1F1B09FF1F2109FF1F00
:102570002C09FF1F0010004010B5002901D001F008
:10258000D3FC10BDF7B5604B01919978A1239B0056
:102590004B435E4A060014681022E418D6235B0001
:1025A000E0583623FF33E35C00279343222B41D1CD
:1025B000574B0F3A1A600760012501F095FD019B0A
:1025C0001880E8235B00E35C002B01D0B34258DDA8
:1025D0000023504FFB70AD33FF33E3581A68002AD5
:1025E00003D09B88DB439B071DD03823FF33E35C7C
:1025F000002B18D09B235B00E35C002B13D1D1335D
:10260000FF33E35CB3420EDAA4235B00E15AE01827
:10261000090A023101F078FC23000122FE33013E59
:1026200001351A87FA70E8235B00E35C002B2AD09F
:10263000A8B2FEBD03683D00002BBED081880430E7
:10264000090A023101F060FCD6235B00E3581F60E9
:10265000B2E72300B133BA00FF33985801378188BD
:102660000430090A023101F04FFCE8235B00E35C0F
:10267000BB42EEDCE822F61AED1800235200A35408
:10268000A6E70027F1E7200001F0DEFC00281FD0BC
:10269000002E1DDD7319882647190193B60020000E
:1026A00001F04AFB5A3080002018406801358188CB
:1026B0000430090A023101F027FC200001F04CFC33
:1026C000A3590133A351BD4202D0019B9D42E6D1E3
:1026D000114BE35C002BABD095239B00E35C002BFC
:1026E000A6D00E4BE15A0029A2D00D4AA35C994214
:1026F00002D90133A3549BE700231A212000A354DD
:1027000001F09AFA94E7C046300DFF1F3409FF1F0D
:1027100000140340E010FF1F5A0200007202000084
:102720005E0200000D4970B54A6E0D4CD2038B69F4
:10273000D20BA24206D80B4D0224AA4204D901F0C2
:10274000ABFA70BD02246442E21815007E242540D5
:102750002242F4D0A3432B438B61F0E700F000400A
:102760000A200000FC1C0000F8B51D4B1D4F1A7814
:10277000002A10D1BA7B002A02D101321A7003E07C
:10278000032AFAD0022AF8D001F016FB0022012019
:10279000154B1A70F8BD154B154D1C68154B9E78DE
:1027A00001232B702878C0B200F0A2FBBB7B002B6A
:1027B0000BD101F0D9FBA1239B007343E4188323C1
:1027C0009B00E41823782B70E4E7032B02D101F07F
:1027D000A3FBF0E70020022BDCD101F00DFBEAE7C0
:1027E0001C09FF1FA60BFF1F2309FF1F3409FF1F32
:1027F000490AFF1F300DFF1FF0B587B00EAD2F78CF
:102800000FAD2D780593AC46634614000E4D0CAA0F
:1028100012782E7803930D9B009201932200059B62
:10282000029701F0C1FA2E70012C01D0042C08D1BE
:10283000802206498B889343054A1278D2011343BC
:102840008B8007B0F0BDC0461C09FF1F6C11FF1F35
:102850007809FF1F0B001B3B70B504003020E02BF4
:102860000DD81300E025493BFF3B9BB2ED00AB4286
:1028700005D8034B200019825A8201F08DFA70BDF1
:102880008410FF1F10B501F0CFFB054B00205B68E3
:10289000052B04D9034A5268D20200D4980810BD0F
:1028A00000100040FCE100E070B501F04DFB0D4B65
:1028B0001B68FC33DC691D6AFFF7E4FF641984427E
:1028C00004D2094B01241B68002B07D004220024EA
:1028D000064B1A70064A93690133936101F014FCA8
:1028E000200070BD1465FF1F9809FF1F2309FF1FFB
:1028F000FC0FFF1F70B50C4D2B68FC335C6A01F0B8
:1029000023FBFFF7BFFF2B680025FC339B6AE3180E
:10291000834204D2054B1B68AB4200D1051B01F07A
:10292000F3FB280070BDC0461465FF1F9809FF1F08
:10293000D722044B92009B5810B5002B00D098472B
:1029400010BDC0460000FF1F10B501F0D3F8FFF71F
:10295000EFFF2749274BCA6D274C1A4084235B00A1
:102960001343CB65254B1B68186A01F0E5FA244B2D
:10297000244A1A60244B254A1A60A022244B520094
:102980001A60244B187801F02FFA2000224901F038
:102990001BFB0023A3600233A360204B204923606C
:1029A00003232048A36001F00FFB10221E4BFF20E1
:1029B0001A60802252031A60802292031A608022D9
:1029C00012041A6001F0F0FA012001F045F9FA2032
:1029D000400001F079FA582001F0BEF9134801F0E7
:1029E00063F9012001F0C8F9072001F0FDFA10BDDC
:1029F00000F0004000FEFEFF141000401465FF1FB1
:102A0000000003400180063DBC0003403408000084
:102A1000A40003404A0AFF1F71020000C30900001E
:102A2000FFFF3F002810004000E100E0307500008B
:102A3000674E336888331B6883F3088801F094F984
:102A4000644A6549136800200B401360634B644A75
:102A50001B68934200D1A6E001F046FA0221614AC8
:102A600013688B431360FFF76FFF5F4B5F4C187861
:102A7000C0B201F011FB0023A3600233A3605C4BE2
:102A80000120236001F058FA0323A36001F00CFA3F
:102A9000040001F0C9FA050001F006FA554B186070
:102AA00001F00AFA544B1968621A531EA14200D26F
:102AB00013008022D203934201D39B029B0A326807
:102AC000D16AC90700D471E04C491C0C09689BB25B
:102AD0004C4359432402090A641803264849FC322E
:102AE00093680A6847489B1A474A0768126847492B
:102AF0009B18474A9A1833409208DB190A60036012
:102B0000042B03D9013233400A6003600E68414947
:102B1000A619300001F078F93F4F3E493B68C318D1
:102B20003B603000019301F0B7F93C4E3068081863
:102B300038493060884205D9019B01333B6001F080
:102B4000ABF9316001F088FA354B1B78002B0DD0C2
:102B500001F06AFA334B621B196812188A4232D2AA
:102B60004919091B091A304801F02EFA2F4E337A01
:102B7000002B0ED001F058FA621BF1681218914236
:102B800024D94919091B091A294801F01DFA002303
:102B90003372284B83F3088801F076F8002001F0A7
:102BA000A3F901F0A1F801F09FF95CE7DC019900BD
:102BB0000234641A5900641A09214B438033CB4014
:102BC000A408E41889E7FA218900CCE71A49DBE771
:102BD0001465FF1F1CF00040FFFFC1FF0C0AFF1F20
:102BE000B641210310000040490AFF1F14100040A5
:102BF000C3090000100AFF1F340AFF1F380AFF1F15
:102C0000200AFF1F280AFF1F1C0AFF1F240AFF1F9C
:102C1000C4090000710200006008FF1F2C0AFF1F9A
:102C20001C09FF1FE408FF1F00100040740BFF1F6A
:102C30003C10004000000020DC050000A022054BF5
:102C400092009B5810B5002B01D0984710BD01F0A1
:102C50001BFAFBE70000FF1FA122054B92009B58C7
:102C600010B5002B01D0984710BD01F00DFAFBE71D
:102C70000000FF1FA222054B92009B5810B5002BAD
:102C800001D0984710BD01F0FFF9FBE70000FF1FDE
:102C9000A322054B92009B5810B5002B01D09847FA
:102CA00010BD01F0F1F9FBE70000FF1FA422054B66
:102CB00092009B5810B5002B01D0984710BD01F031
:102CC000E3F9FBE70000FF1F70B501F0ADF94F4BD2
:102CD000186000F0F9FF0400C30702D401F00CFAF9
:102CE00070BD00224A4B1A604A4B187801380428FC
:102CF00029D800F075FF0320181C2400200001F0E3
:102D0000BBF80128ECD0444C2378042B6ED100F0A2
:102D10007BFF0028E4D001F037F9582001F01CF8BF
:102D200002232370DCE7200001F02EF8E9E7200001
:102D300001F07AF8E5E7200001F04EF8E1E7200025
:102D400001F09AF9DDE701F07FF80500012808D1CC
:102D5000324B1B78053B012B03D82000FFF76EFF99
:102D6000D1E72D4B1B78022B01D0052B20D1022D52
:102D700028D12B4B9B7BAB431CD12000FFF76CFF72
:102D8000264B18780128BED16405BCD424492522DD
:102D90004B7B034205D1233A13405A425341263319
:102DA0001A000B7D9342AED9322000F085FFAAE7CE
:102DB000022D07D1194B1B78052B11D12000FFF7ED
:102DC00059FFDDE7012D0BD1012B03D12000FFF7C7
:102DD0005FFF98E7062B03D12000FFF767FF92E71C
:102DE000200001F051F9022D8DD1C9E7032B04D148
:102DF0000C4B987C00F040FF72E7072B00D06FE788
:102E0000094B987B00F010FF6AE7C0469C09FF1F42
:102E10009809FF1F9009FF1F2309FF1F1C09FF1FAF
:102E2000A60BFF1FBC0BFF1FD40BFF1FFA210A4B81
:102E30000A4A49001A640A4A5A500A4A04395A503E
:102E4000094A08319A64094A5A50094A5C315A5071
:102E5000084ADA667047C0460000FF1FF927FF1FC7
:102E6000F528FF1FA928FF1FD923FF1F6927FF1F70
:102E7000791EFF1F4D1EFF1F10B500F099FE10BDFB
:102E8000F7B50B0CFF270122009300233C001E0026
:102E90001D009446019089B262469A401000084095
:102EA00018413618B6B2FF2F02D1012E00D19FB2C1
:102EB000009802401A41AD18ADB2FF2C02D1012D8D
:102EC00000D19CB20133102BE6D10320012E07D193
:102ED000012D04D1019B2401E4191C700138FEBDB1
:102EE000102EFCD10238102DF9D00230F7E7000087
:102EF0008023F7B59C46264B264F01932649274A47
:102F0000274D284C284B02281AD1604638600868A3
:102F1000264E3040802636033043086001990978F8
:102F2000002909D11660224A2A60224A2260E02242
:102F300019689143A03A1BE08021C9021160F2E7B1
:102F400066463E600F68194E3E408027FF023E43B2
:102F50000E600199097800290DD1176001280ED162
:102F6000154A2A60154A2260E02219689143C03A46
:102F70000A431A60F7BD802189021160EEE7E02163
:102F80000F4A02432A600F4A22601A688A43F0E718
:102F90004B0AFF1FE0000340D800034090000340AD
:102FA000000003405000034040000340FFFFE3FFE8
:102FB0000280063D804508220180063D8066082289
:102FC0000080069880550822F8B51E4B80261A68A6
:102FD000002014003440324232D11A681A4F324372
:102FE0001A6001223B68063093433B6000F0A4FF67
:102FF0000122164D2B681E432E603B680A261343A0
:103000003B608027BF00124B1B683B4211D1013E41
:10301000F6B2FF2E09D17E220E4B1C682B68E40B02
:103020001440934323432B6005E0082000F084FF05
:10303000E9E7002EEFD180222B68600893432B60D4
:10304000F8BDC046C4F000405CF0004018F00040FD
:1030500068F0004060F0004010B500F065FE01210E
:103060005820034A00F0D8FEFFF7AEFF10BDC0465F
:10307000600AFF1F10B578220021034800F064FEAB
:1030800000F0DAFE002010BD1C68FF1F70B50400C0
:1030900000F05AFF00230C200B4A010059438D1801
:1030A000515C00290DD0A14208D1012300246B708E
:1030B00000F062FF01F028F8200070BD01330A2BF8
:1030C000EBD11224F6E7C0461C68FF1F70B5040060
:1030D00000F03AFF002319001D000D4A1078002867
:1030E00006D0A0420CD1557001310C320A29F5D11D
:1030F000002B0AD100F0A0FE01F006F8002070BD00
:103100005078461EB0411B18EEE700F035FFF3E79C
:103110001C68FF1FF7B504000C20002384460E4DE9
:10312000019267465F43E85D7E19A04212D00028F5
:103130000BD10A4B9C4662461B7808331370019BE7
:1031400070707C557160B360FEBD01330A2BE8D10D
:103150000320F9E70720F7E71C68FF1F1868FF1F27
:103160008020F8B5484BC0051B68C1248360474BDD
:10317000FF251A68012313434361454BA4001A68D5
:10318000444B40211A60444B1A68444B1A60444B2C
:103190001A59AA431A51C52292009E58AE43314390
:1031A000802699509F583F49F6010F403E439E505C
:1031B0009E5880273602360A3043985080201A598C
:1031C00000020A4002431A5104341A59364E3F0491
:1031D000324080263A431A511A5936061202120A10
:1031E00032431A5108341A5980260A4002431A51B0
:1031F000C32292009F58B446AF4337439F509F5815
:10320000294E0F4007439F509F5837408026360471
:10321000374380269F509F5836063F023F0A374368
:103220009F50C0221F59AF433A431A511A591202F4
:10323000120A1643C6221E5192009C58AC436546A2
:103240002C439C509C5800250C4020439850C7208C
:1032500080001A58154C1140C02212020A431A501D
:10326000134B1B78DB08AB4201DC0020F8BD237850
:10327000002B06D0A368002B00D0984701350C34F2
:10328000EEE71220F2E7C0461444FF1F1044FF1F70
:10329000B0F000401468FF1FB4F000401068FF1F3A
:1032A00000E100E0FF00FFFFFFFF00FF1C68FF1FC1
:1032B0001868FF1F030010B51F2809D80722002037
:1032C0001340072404490A78A24313430B7010BD2E
:1032D00000230620F5E7C0461868FF1F054B064986
:1032E0001B780A6805485B0702401B0B134300204C
:1032F0000B6070471868FF1F1CF00040FFFFC1FF04
:1033000070B50C25FFF7EAFF0A4B1C780A4BE4085E
:103310006543ED18002C01D1200070BD2B78002BE7
:1033200006D06B68002B00D09847013C0C3DF1E7BC
:103330001220F2E71868FF1F1068FF1F1FB5002159
:1033400002220B0001910091052000F045FE0223AE
:103350000B490A681A42FCD120230393039B5A1E8F
:103360000392002BFAD1074A1368002BFCDA0B24D6
:103370006C442000012100F0CFFC207804B010BD87
:1033800090C8004000C8004013B504000A4B0193E8
:10339000019B002B01D1112016BDFFF7CFFF2300A9
:1033A0000340044205D0052000F0C6FD019B013B0F
:1033B000EDE71800F0E7C046FFFFFF0707B500F094
:1033C000C3FD80220821D205936A0191002B01D10F
:1033D0000739916202210C4A11600199481E01903F
:1033E0000029FAD103311160053101910199481E7C
:1033F00001900029FAD11160002B02D18022D20560
:10340000936200F081FE07BD00C00040F0B52D4C76
:1034100089B02378002B4FD1FEF7CEFA02232A4F32
:1034200003903A681A42FCD120230693069B5A1E49
:103430000692002BFAD1254E3368002BFCDA0120CE
:10344000FFF7A2FF011E02D0112009B0F0BD03005A
:1034500003220190009005AD9F2000F0BDFD0321E7
:10346000280000F059FC02233A681A42FCD12023BC
:103470000793079B5A1E0792002BFAD13368002B43
:10348000FCDA0120FFF780FF0028DDD10398FEF76A
:10349000A7FAAA786B7811041B020B4329780B4317
:1034A00063601300113B0A49052B07D801239340A1
:1034B000A3600B60012323700020C6E780231B0359
:1034C000F6E7C046FC43FF1F90C8004000C800401C
:1034D0009808FF1F1E4B30B55A6818781D4B85B0F1
:1034E000D31859424B4101210093002300F00CFCFA
:1034F000194B1A4A02259A6300221A6510325A653E
:103500008022C4219D65164B1648D202DA678900D5
:103510004258154B80241A4080231B041343435008
:10352000642341200393E40500F006FA402000F0F4
:1035300003FA6562039D6B1E0393002DFAD10323EA
:103540006362FFF73BFFA562FFF760FF05B030BD88
:103550000844FF1F95FFFEF700C80040050001FF6B
:1035600004E100E000E100E0FFFF00FFF0B585B0FE
:103570000700FEF721FA022305002D4C22681A42AB
:10358000FCD120230093009B5A1E0092002BFAD1FD
:10359000284E3368002BFCDA0120FFF7F5FE0028E7
:1035A00003D01124200005B0F0BD234B236002237B
:1035B00022681A42FCD120230193019B5A1E0192DA
:1035C000002BFAD13368002BFCDA0120FFF7DCFE78
:1035D0000028E6D1194B1F60022322681A42FCD151
:1035E00020230293029B5A1E0292002BFAD13368C9
:1035F000002BFCDA0120FFF7C7FE0028D1D1104BC9
:103600002360022322681A42FCD120230393039BE8
:103610005A1E0392002BFAD13368002BFCDA0120EA
:10362000FFF7B2FE041EBCD12800FEF7D9F9B9E7B6
:1036300090C8004000C8004001000006A8C8004033
:103640000180000110B50020FFF790FF10BD0000C1
:1036500010B5064B18705960FFF73CFF002113208E
:10366000034AFFF757FD002010BDC0460844FF1F66
:10367000D534FF1FF0B5040085B003920291FEF728
:103680009BF9882263035B0B52051A438023DB05F9
:103690009D6A8023274F0092BA68002601901B0381
:1036A0009A420CD9F82326001B041E401C4206D067
:1036B0008022214B52025E6219680A431A60002D73
:1036C0000BD100F041FC02221C4B1A608023DB0569
:1036D0005A62013A9A6200F017FD0023039A93425E
:1036E00020D1002D0AD100F02FFC144B03221D60C5
:1036F0008023DB055A629D6200F006FD8023BA68D4
:103700001B039A4208D9002E06D000220A4B0C490E
:103710005A621A680A401A600198FEF761F900209F
:1037200005B0F0BD009A0299D2181278CA5401333C
:10373000D4E7C046FC43FF1F00C8004000C0004063
:10374000FFFFFEFFF0B587B0029103920400FEF781
:1037500033F9019000F0F8FB802302250122234E6B
:10376000DB0535605D629A6200F0CEFC204F3B685D
:103770002B42FCD120230493049B5A1E0492002B5D
:10378000FAD11C4D2B68002BFCDA0120FFF7FCFD61
:10379000002802D0112007B0F0BD2000039A029942
:1037A00000F072FB022304003A681A42FCD1202385
:1037B0000593059B5A1E0592002BFAD12B68002B0E
:1037C000FCDA0120FFF7E0FD051EE3D100F0BCFBB1
:1037D00080230322DB0535605A629D6200F094FC71
:1037E0000198FEF7FDF8E0B2D5E7C04600C0004002
:1037F00090C8004000C80040F0B5802489B00600A1
:10380000FEF7DAF8E405A36A02250393029000F0BC
:103810009BFB0123304F3D606562A36200F074FCA6
:103820002E4C23682B42FCD120230593059B5A1E66
:103830000592002BFAD12A4D2B68002BFCDA0120CF
:10384000FFF7A2FD002803D01124200009B0F0BD2D
:10385000244B2360022322681A42FCD120230693C2
:10386000069B5A1E0692002BFAD12B68002BFCDA1D
:103870000120FFF789FD021EE6D11B4B03211E60CC
:10388000030001900090202000F0A6FB0223226894
:103890001A42FCD120230793079B5A1E0792002B44
:1038A000FAD12B68002BFCDA0320FFF76DFD041E14
:1038B000CAD100F049FB80230322DB053C605A6239
:1038C0009C6200F021FC039B002B01D1FFF776FDE9
:1038D0000298FEF785F8B8E700C0004090C80040A5
:1038E00000C800400100000694C8004007B500026F
:1038F00001910422000A01A9FFF724FF0EBD000078
:1039000073B5050005240B4AA3005B429B18196898
:103910006B46DE1D3000FFF7B3FA022804D133787E
:103920002B55013CEFD276BD052CFCD00128FAD1F5
:103930000230F8E7140900111F2807D8012380225C
:103940008340D20591680B43936070473F2808D8A5
:103950000123802220388340D20551690B435361F3
:10396000F3E75F28F1D80123802240388340D20555
:10397000116A0B431362E8E71F2807D80122802150
:103980008240C9058B6893438B6070473F2808D8F5
:103990000122802120388240C9054B6993434B6145
:1039A000F3E75F28F1D80122802140388240C90521
:1039B0000B6A93430B62E8E71F2810D880230200AC
:1039C000DB05153A1968012A06D8202291431960AF
:1039D00019680A431A60704701228240F6E73F28BF
:1039E00011D880230200DB05353AD968032A06D8AE
:1039F00010229143D960D9680A43DA60EBE70122CB
:103A000020388240F5E75F28E5D842238022181A43
:103A1000413B8340D205516A99435162516A0B433D
:103A20005362D8E710B50400012813D1A022184929
:103A300092050B685B015B0913430B60154B164A3B
:103A400019681140154A0A431A60402219680A434E
:103A50001A6010BD0028FCD101000A2000F0ECFA29
:103A600021000B2000F0E8FAC0220A4B92001968EE
:103A70000A4340211A601A688A431A60B022044936
:103A800012060B685B015B0913430B60E1E7C0465C
:103A900014F000401CF000407F00FEFF80FD01009C
:103AA00072B6074A1368013313600422054B1A608B
:103AB0000023054A13608022D2055360FEE7C0460A
:103AC0007808FF1FC0F00040C4F0004005490B68B3
:103AD000002B05D1044A0A6004490A60044A1360B5
:103AE0007047C046140AFF1F841E0000380AFF1FDB
:103AF000C4F000400023034A1360034A1360034AE2
:103B00001360704754F0004040F1004044F1004021
:103B1000002310B5184C8AB0009301932378012B31
:103B200027D06946012000F077FA002817D1009BC2
:103B300012490293019B06AA0393114B02A81B682A
:103B40000493104B1B68059300F0D6F810220E4921
:103B500006A800F061F8002804D1FF23237000209C
:103B60000AB010BD0123094A074902A8237000F0DA
:103B7000C3F80120F4E7C0461865FF1F10290011A3
:103B8000082900110C290011202900111C65FF1FB4
:103B900013B501246946012000F03EFA034B00945E
:103BA0000193FFF7B5FF200016BDC046BB0B000018
:103BB00010B5FFF79FFFFFF7EBFF002802D0024B85
:103BC000984710BDFEE7C046E1A2000002B471466E
:103BD00049084900095649008E4402BC7047C04656
:103BE00002B4714649084900095C49008E4402BC90
:103BF0007047C04603B47146490840004900095A5D
:103C000049008E4403BC704701B40248844601BC9D
:103C1000604700BF01D7000001B40248844601BCE0
:103C2000604700BFCD4C010001B40248844601BC8E
:103C3000604700BFC1F7000001B40248844601BCE0
:103C4000604700BF53B9000001B40248844601BC7C
:103C5000604700BF8B52010001B40248844601BC9A
:103C6000604700BF6911010001B40248844601BCED
:103C7000604700BFE927000001B40248844601BC48
:103C8000604700BF4DF9000001B40248844601BC02
:103C9000604700BF7997000001B40248844601BC28
:103CA000604700BFD1AE000001B40248844601BCA9
:103CB000604700BF8D11010001B40248844601BC79
:103CC000604700BF6137010001B40248844601BC6F
:103CD000604700BFBD0B010001B40248844601BC2F
:103CE000604700BFB352010001B40248844601BCE2
:103CF000604700BF8552010001B40248844601BC00
:103D0000604700BFDD3F000001B40248844601BCAB
:103D1000604700BFC56D010001B40248844601BC84
:103D2000604700BF3D71010001B40248844601BCF8
:103D3000604700BFED68010001B40248844601BC41
:103D4000604700BFD9B0000001B40248844601BCFE
:103D5000604700BFB70E000001B40248844601BCB2
:103D6000604700BF7912010001B40248844601BCDB
:103D7000604700BFC9A9000001B40248844601BCE5
:103D8000604700BFE512010001B40248844601BC4F
:103D9000604700BF0934010001B40248844601BCF9
:103DA000604700BF116E000001B40248844601BCA8
:103DB000604700BF9D6A000001B40248844601BC10
:103DC000604700BFA9D8000001B40248844601BC86
:103DD000604700BF51B8000001B40248844601BCEE
:103DE000604700BFF535010001B40248844601BCBC
:103DF000604700BFEDA5000001B40248844601BC45
:103E0000604700BF19FA000001B40248844601BCB3
:103E1000604700BF090E000001B40248844601BC9F
:103E2000604700BF0167010001B40248844601BC3D
:103E3000604700BF0534010001B40248844601BC5C
:103E4000604700BFADAE000001B40248844601BC2B
:103E5000604700BFDD0C010001B40248844601BC8C
:103E6000604700BFC1A5000001B40248844601BC00
:103E7000604700BFE94C010001B40248844601BC20
:103E8000604700BF0134010001B40248844601BC10
:103E9000604700BF9573010001B40248844601BC2D
:103EA000604700BF090E000001B40248844601BC0F
:103EB000604700BF156B010001B40248844601BC95
:103EC000604700BFC166010001B40248844601BCDE
:103ED000604700BF8512010001B40248844601BC5E
:103EE000604700BFF9ED000001B40248844601BC00
:103EF000604700BF016C010001B40248844601BC68
:103F0000604700BF8944000001B40248844601BCF8
:103F1000604700BFC115010001B40248844601BCDE
:103F2000604700BF75F8000001B40248844601BC38
:103F3000604700BFE9D4000001B40248844601BCD8
:103F4000604700BF0189000001B40248844601BCFB
:103F5000604700BF75A9000001B40248844601BC57
:103F6000604700BF5976010001B40248844601BC95
:103F7000604700BFE9F6000001B40248844601BC76
:103F8000604700BF21A9000001B40248844601BC7B
:103F9000604700BF6DF6000001B40248844601BCD2
:103FA000604700BFCDB5001101B40248844601BC92
:103FB000604700BFED6B010001B40248844601BCBC
:103FC000604700BF6D0B010001B40248844601BC8C
:103FD000604700BF2D6C010001B40248844601BC5B
:103FE000604700BF496D010001B40248844601BC2E
:103FF000604700BFF90D010001B40248844601BCCE
:10400000604700BF2144000001B40248844601BC5F
:10401000604700BFBD5C010001B40248844601BC9A
:10402000604700BFE1AC000001B40248844601BC17
:10403000604700BFC95C010001B40248844601BC6E
:10404000604700BF25A2001101B40248844601BCAC
:10405000604700BF71B0000001B40248844601BC53
:10406000604700BFD544010001B40248844601BC4A
:10407000604700BF8D82000001B40248844601BC45
:10408000604700BFF935010001B40248844601BC15
:10409000604700BFE917010001B40248844601BC33
:1040A000604700BF8914010001B40248844601BC86
:1040B000604700BF85C1000001B40248844601BCCE
:1040C000604700BFE90B010001B40248844601BC0F
:1040D000604700BF0D52010001B40248844601BC94
:1040E000604700BF8937010001B40248844601BC23
:1040F000604700BFCD0C010001B40248844601BCFA
:10410000604700BFDD0A010001B40248844601BCDB
:08411000604700BF9DA90000FB
:10411800020000006EBE00110100000080BC00110A
:10412800020000006ABE0011010000005841FF1F94
:104138000200000088BC0011010000009062FF1F0F
:104148000200000068BE0011030000000462FF1FA7
:1041580012000000020000006EBE00110100000005
:10416800C8BC0011020000006ABE00110100000076
:10417800C5BC001102000000D2BC00110300000001
:104188003F62FF1F0200000068BE0011030000002C
:104198005462FF1F020000006ABE00110100000007
:1041A800C4BC001102000000D0BC001103000000D4
:1041B8001562FF1F0200000068BE00110300000026
:1041C8003662FF1F020000006EBE001101000000F1
:1041D80008BD0011020000006ABE001101000000C5
:1041E800A142FF1F020000001ABD001101000000DB
:1041F80003BD0011020000006ABE001101000000AA
:10420800A042FF1F0200000018BD001101000000BD
:104218005C62FF1F020000006ABE0011010000007E
:104228009F42FF1F0200000016BD001101000000A0
:10423800F3BC0011020000006ABE0011010000007A
:104248009E42FF1F0200000014BD00110100000083
:10425800EEBC0011020000006ABE0011010000005F
:104268009D42FF1F0200000012BD00110100000066
:10427800E9BC0011020000006ABE00110100000044
:104288009C42FF1F0200000010BD00110100000049
:10429800E4BC001102020202020200000000000059
:1042A800161500009D4B0011634B00115CBD0011F9
:1042B80090011D0018001800FFFF07010203040504
:1042C80006020106000000000000000000000000D7
:1042D80000000000000000000000000000000000D6
:1042E80003000000020000006EBE00110100000083
:1042F8007CBD0011020000006ABE00110100000030
:104308005C43FF1F0200000086BD00110100000091
:104318008A62FF1F0200000068BE0011030000004F
:10432800F464FF1F020000006ABE001101000000D3
:104338005C43FF1F0200000084BD00110100000063
:104348008C62FF1F0200000068BE0011030000001D
:10435800EC64FF1F12A6A6A60000000000000000E3
:10436800161500000001000000000111FFFF000009
:104378005048593600000000000000000B000500FE
:10438800F0000000B4000028002800283075A000C4
:10439800A000A000A00000080008E001F000100044
:1043A80010001000100010001000500050005000C5
:1043B80010001000D0070000000000000F000100EE
:1043C8000500307507001000010081FF00000000A3
:1043D800FF0000000D74001115720011A56F001187
:1043E800FFFF0100FF000000299E0011A59B00119E
:1043F800BD9A001100000000000000000000080045
:10440800040000003B0001085902E001882128004F
:10441800FF000000020000006EBE00110100000055
:1044280034BF0011020000006ABE00110100000044
:104438009944FF1F0200000066BE00110100000041
:10444800D468FF1F020000006ABE001101000000CE
:104458009844FF1F0200000064BE00110100000024
:104468009644FF1F020000006ABE00110100000010
:104478009444FF1F0200000062BE0011010000000A
:104488008C44FF1F180018001D0090010200000353
:1044980002020000020000006EBE001101000000D0
:1044A80048BF0011020000006ABE001101000000B0
:1044B800DC44FF1F0200000060BE00110000000085
:1044C800000000000200000068BE001103000000A8
:0644D800F468FF1F20FF45
:040000051FFF184180
:00000001FF
